:020000040800F2
:100000000011002001010008DF370008C1280008A6
:10001000DD370008410F0008AD6100080000000056
:10002000000000000000000000000000A5470008DC
:100030008F1A0008000000003D3D0008A54A000896
:100040001B0100083D3B00081B0100081B010008C4
:100050001B0100081B0100081B0100081B01000810
:100060001B0100081B0100081B0100081B01000800
:100070001B0100081B010008491500081B010008AE
:100080001B0100081B0100083D0700081B010008B8
:100090001B0100081B0100081B0100081B010008D0
:1000A000154B0008F54B00081B0100081B01000858
:1000B000F94B0008E94E0008455100081B010008F3
:1000C0001B0100081B0100081B0100081B010008A0
:1000D0001B010008A55C00081B0100081B010008AB
:1000E0001B0100081B0100081B010008DFF80CD0F1
:1000F00000F0E6FA00480047817200080011002075
:100100000648804706480047FEE7FEE7FEE7FEE7B1
:10011000FEE7FEE7FEE7FEE7FEE7FEE7C54A00086A
:10012000ED0000082DE9F0410024061B254671F181
:10013000000605DA01240027D0EB070067EB010178
:10014000161E73F1000605DA0027D2EB070201251F
:1001500067EB030300F0D0F986460E4617469C462F
:10016000AC4204D00025D0EB050E65EB010624B1AE
:100170000020D2EB000760EB030C704631463A4694
:100180006346BDE8F08140EA01039B0703D009E024
:1001900008C9121F08C0042AFAD203E011F8013B73
:1001A00000F8013B521EF9D2704780EA010210B5F7
:1001B00002F00043400022D04A001FD0010E01EBA4
:1001C0001261C0F35600C2F3560240F4000042F43C
:1001D0000002A0FB022000047F39140400D0401C60
:1001E00050EA124001D44000491EC2B20C0604EB92
:1001F000D010401C4008802A02D003E0002010BD2F
:1002000020F00100002900DA0020184310BD2DE97C
:10021000FE4F81EA030404F0004421F00041009401
:100220004FF0000B23F0004350EA01045ED052EA85
:1002300003045BD0C3F30A54C1F30A552C44A4F25F
:10024000F3340194A0FB0254C1F3130141F4801173
:10025000C3F3130343F4801301FB024400FB034E7A
:10026000840A970A44EA815447EA8357A4FB076843
:1002700002958D0A05FB07854FEA932C04FB0C546D
:100280002705029D4FEA065847EA1637B5EB0805E1
:100290006EEB070C870E920E47EA811742EA831233
:1002A000A7FB0201B6EB0B0164EB00042B0D43EA44
:1002B0000C335E1844EB1C50DA465146E7FB020152
:1002C000C5F313044FEA0B3343EA14534FEA0432E5
:1002D000019C43EA0603A4F10C040294009CCDE9BE
:1002E00000B400F09FF903B0BDE8F08F0020014694
:1002F000F9E72DE9F04D81EA030404F0004B21F009
:10030000004514464FF0000A23F0004150EA050270
:1003100020D054EA01021DD0C5F30A570246C5F3A6
:100320001303C1F31300C1F30A5640F4801543F4DC
:100330008013A7EB0608101BD64608F2FD3873EBB6
:10034000050002D308F1010801E092185B41B8F101
:10035000000F03DA00200146BDE8F08D00204FF4C5
:100360008011064684460EE0171B73EB050705D384
:10037000121B63EB050306434CEA010C49084FEAE4
:10038000300092185B4150EA0107EDD152EA0300B8
:1003900012D082EA040083EA0501084305D0101B4D
:1003A000AB4106D20122002306E000224FF00043B9
:1003B00002E06FF0010253101AEB06004CEB0851FB
:1003C00010EB0A0041EB0B01BDE8F04D00F01BB94A
:1003D00070B521F0004303430CD0C1F30A5500244B
:1003E000D5EB040564EB0403D617AD1AB34102DB69
:1003F0000020014670BD201841EB025170BDC10FB5
:1004000080EAE0700844CA079623002100F0CDB8C6
:1004100096230022114600F0C8B80EB5C10F80EA3D
:10042000E0700844CA07002140F233438DE80E0013
:100430000A460B4600F0F6F803B000BD0EB540F2D8
:10044000334102910021CDE900110A460B4600F02C
:10045000E9F803B000BD00F0004220F00040C10DFB
:10046000C0F3160040F400007F2901DA0020704735
:10047000962903DCC1F19601C84001E09639884015
:10048000002AF4D04042704770B5C1F30A5201F01F
:1004900000450024C1F3130140F2FF3341F4801101
:1004A0009A4201DA002070BD40F233439A42A2F230
:1004B000334203DC524200F05FF800E090402C43EE
:1004C000F1D0404270BDC1F30A5210B5C1F313011F
:1004D00040F2FF3341F480119A4201DA002010BD4E
:1004E00040F233439A42A2F2334203DC524200F01C
:1004F00043F810BD904010BD2DE9F05F0546002087
:1005000092469B4688460646814640241BE0284684
:1005100041464746224600F02FF853465A46C01A35
:10052000914110D311461846224600F016F82D1AB4
:1005300067EB01084F4622460120002100F00DF82C
:1005400017EB00094E41201EA4F10104DFDC4846F0
:1005500031462A464346BDE8F09F202A04DB203A74
:1005600000FA02F1002070479140C2F1200320FA06
:1005700003F3194390407047202A04DB203A21FA04
:1005800002F00021704721FA02F3D040C2F12002AC
:1005900091400843194670470029A8BF7047401C86
:1005A000490008BF20F00100704710B4B0FA80FC89
:1005B00000FA0CF050EA010404BF10BC704749B1C6
:1005C000CCF1200421FA04F411FA0CF118BF012136
:1005D00021430843A3EB0C01CB1D4FEA00614FEA16
:1005E000102042BF002010BC704700EBC3501044E5
:1005F0000029A4BF10BC7047401C490008BF20F070
:10060000010010BC704710B5141E73F1000408DA25
:10061000401C41F1000192185B411A4301D120F0C6
:10062000010010BD2DE9F04D92469B4611B1B1FA83
:1006300081F202E0B0FA80F220329046FFF78DFF9F
:1006400004460F4640EA0A0041EA0B0153465A4667
:10065000084313D0114653EA010019D0C8F14002F3
:100660005046FFF789FF05460E465046594642461A
:10067000FFF773FF084305D0012004E02046394608
:10068000BDE8F08D0020054346EAE0762C43374371
:100690000A986305E40AA0EB08000022FD0A44EA78
:1006A00047540A3002D500200146E9E70105101938
:1006B0006941DDE9084500196941BDE8F04DA2E74F
:1006C000064C074D06E0E06840F0010394E807009F
:1006D00098471034AC42F6D3FFF70CFDCC930008DA
:1006E000EC93000870B58C1810F8015B15F0070347
:1006F00001D110F8013B2A1106D110F8012B03E0BB
:1007000010F8016B01F8016B5B1EF9D12B0705D4C2
:100710000023521E0DD401F8013BFAE710F8013B0B
:10072000CB1A921C03E013F8015B01F8015B521E27
:10073000F9D5A142D8D3002070BD000070B54F4C50
:100740004FF490652946204600F01BFA002866D039
:100750002946204600F0A8F849490888401C08802E
:100760000121204600F0ECFA464942F21072B1F83D
:100770005000904202D2401CA1F8500006F060FFE9
:1007800005F076F8404DB5F91410B5F9120005F0F2
:100790003FFE3E4CA5F856002080A16820468847C1
:1007A000A088A5F8580003F083F807F049F8384E00
:1007B000384C3078082833D045F6AC30606042F6CB
:1007C000EF60A06042F2C400E0603348008A2080FD
:1007D000208E6080A16B2F488847208E69882F4C1F
:1007E00008444FF6FF7101EA80006887207A4FF0D5
:1007F000000540071DD501F0D9FA294949F6A24064
:100800000880284840F21A62C188491C89B2C18018
:10081000914204D3A16821F00401A160C58070BD9C
:1008200041F2130060604FF48060A06040F61B50FE
:10083000CAE730780A281BD2DFE800F01A0616054E
:100840000A050D1A1114EAE7BDE8704005F084BFEF
:1008500007F01AFF08E0BDE8704002F073BD06F033
:1008600001FB01E007F044F9BDE8704007F040B932
:1008700000F0FEFB84F8B65070BD0000002401407B
:10088000FC0600203C01002060000020180700202A
:10089000F3060020D8000020EC0100209802002080
:1008A000442C0140340900206FEA11210160704797
:1008B0000029816802D041F0010101E021F001012D
:1008C000816070470029816802D041F4807101E0A5
:1008D00021F48071816070472DE9F041824E92B021
:1008E000304600F00BF90BA800F039FA01214FF463
:1008F000C06003F0D9FA00248DF831404FF4602035
:10090000CDE90D044FF4A0204FF009080B9001270A
:100910008DF83C808DF830700BA9304600F080F9DE
:10092000724D8DF831408DF830708DF83C700BA908
:10093000284600F075F901231A460F21304600F0D1
:10094000C0F9022201231146304600F0BAF9012312
:1009500003220021304600F0B4F901230422194695
:10096000304600F0AEF9012305220B21304600F09D
:10097000A8F9012306220421304600F0A2F9012340
:1009800007220821304600F09CF9012308220321A8
:10099000304600F096F9012309220A21304600F082
:1009A00090F90121304600F084F90121284600F039
:1009B00080F901231A460521304600F055F901233C
:1009C0001A460621284600F04FF90021304600F073
:1009D000CBF84FF4E041284600F0C6F8012130463C
:1009E00000F0B8F80121284600F0B4F801213046A3
:1009F00000F0A6F80121284600F0A2F801213046B7
:100A000000F09EF90121284600F09AF940F61451B1
:100A1000374804F06EFE12208DF8400002208DF859
:100A200041008DF842408DF8437010A802F004FF99
:100A300001224FF49061304600F0E8F80121304681
:100A4000FFF740FF01213046FFF732FF0121284622
:100A5000FFF72EFF304600F06EF9304600F09FF8A9
:100A60000028FAD1304600F075F9304600F082F8DF
:100A70000028FAD1284600F05EF9284600F08FF8E9
:100A80000028FAD1284600F065F9284600F072F8EF
:100A90000028FAD10121084603F0E2F9154D284655
:100AA00000F08EFD684600F036FE0F4801A94C307C
:100AB0000090114881E811018020CDE904404000F8
:100AC000069080000790202008904FF44050CDE918
:100AD00009046946284600F001FE0121284600F07D
:100AE00063FD12B0BDE8F081002401400028014000
:100AF000002C014008000240A80200200D4910B55A
:100B0000884202D1012144150AE00B49884202D1F2
:100B10000121041504E0094988420AD10121CC03CE
:100B2000204603F0CDF92046BDE81040002103F037
:100B3000C7B910BD0024014000280140003C01401D
:100B40000029816802D041F4801101E021F4801174
:100B5000816070470029816802D041F4004101E0C2
:100B600021F4004181607047826822F4E0420A4328
:100B700082607047014600208968490700D501203E
:100B8000704710B50246002054680B0AC9B20C40E9
:100B90001168194202D0002C00D0012010BD01467E
:100BA00000208968090700D50120704738B5012168
:100BB0001C2003F079F9FF20ADF8000000248DF827
:100BC000034003258DF8025069460D4801F0E8FA0C
:100BD0000120ADF800008DF803408DF80250694601
:100BE000084801F0DDFA2320ADF800008DF803403D
:100BF0008DF802506946044801F0D2FA38BD000071
:100C000000080140000C014000100140002A426829
:100C1000C9B201D00A4300E08A4342607047000035
:100C200010B542680E4B0C791A400B6842EA042258
:100C30001343436083680B4A1340D1E902422243C5
:100C40004C7943EA44031A438260C26A097C22F465
:100C50007002491EC9B242EA0151C16210BD0000D2
:100C6000FFFEF0FFFDF7F1FF70B5072409290AD94F
:100C7000C568A1F10A0606EB4606B440A543B34099
:100C80001D43C56007E0056901EB4106B440A5437B
:100C9000B3401D430561836BC3F30154121B921CC7
:100CA00002EB82041F22A2409343A1400B438363C3
:100CB00070BD826B491E22F4401242EA01518163E9
:100CC000704770B5072409290AD9C568A1F10A0639
:100CD00006EB4606B440A543B3401D43C56007E09C
:100CE000056901EB4106B440A543B3401D430561CE
:100CF0001F23072A09D2446B521E02EB8202934043
:100D00009C4391400C43446370BD0D2A09D2046B8F
:100D1000D21F02EB820293409C4391400C43046338
:100D200070BDC46A0D3A02EB820293409C4391402D
:100D30000C43C46270BD816841F008018160704756
:100D40000029816802D041F4A00101E021F4A00152
:100D500081607047816841F0040181607047002123
:100D60000160017141718160C160012101747047AE
:100D700070B51E4C214694F83800B1F84250062850
:100D80001ED9B4F84A10B4F84C00A1EB000202F1ED
:100D90000902122A04D8FFF751FB0022144B0AE083
:100DA000884204D2FFF74AFB0022124B03E0FFF710
:100DB00045FB0022104BFFF72AFAFFF784FB09E0FE
:100DC00005D12846FFF73AFB0C4A0D4BF3E70D49D6
:100DD00051F82000C5EB45116063B0EB410F03D91A
:100DE000C5EB45104000606370BD0000400400206A
:100DF00000003440000033400000354067666666FE
:100E000066E64B40748B000810B50C4C2078400708
:100E100013D5FFF7ADFF0A49A08E08800848303887
:100E2000018821F010010180001F018841F01001AC
:100E30000180207820F00400207010BD40040020C4
:100E400040040040F0B4184816494FF49677436CBC
:100E500008468A68046815485FEAC25C42F00806E2
:100E6000007822F008054FEA047415D5002C08DB41
:100E7000120714D408B1082811D1BB420FDA8E60D2
:100E800007E012070BD508B1082808D1BB4206DAE3
:100E90008D60F0BC05F0E8BD002CF2DAE8E7F0BCAC
:100EA00070470000980200203C010020F30600205B
:100EB00070B506464089204B204C4FF480710025C8
:100EC00080B362887AB1012A0CD1E188491C89B2C9
:100ED000E1803289914205D36580E580FF2801D009
:100EE000401E708170BD70882288904201D9012215
:100EF00000E00022184601F0DCF97088B188014456
:100F00002088401C80B220808142EBD82580A088B8
:100F1000401C80B2A080F1888842E3D30120608029
:100F2000A58070BDFFE70022184601F0C2F9A58038
:100F3000E58025806580F4E7000C0140B0050020C5
:100F4000FEE70000FCB505464FF6FF7600200C4694
:100F5000ADF8006048F205078DF8040020E000BFFE
:100F600015F8010B8DF8040001A9084602F0C7F836
:100F7000BDF800009DF8041080EA0120ADF80000E3
:100F80005FF00000BDF800100A0402D587EA4101B5
:100F900001E006EA4101401CADF800100828F1DB31
:100FA000641EDDD26946084602F093F8BDF80000E1
:100FB000FCBD00000246002004E000BF12F8013B27
:100FC0001844C0B2491EF9D27047000070B5144AE7
:100FD00085B010880024134901940094039420469E
:100FE0000494138807E00D8B009E35440095CD8B4B
:100FF000019E3544019515889D42F4D0401CC0B235
:101000008028EED3009841110748418084800198E0
:101010004111064881830183818205B070BD0000C3
:10102000FC06002098020020CA050020B804002019
:1010300030B50E4902880A800C4A4388083A13806A
:101040000B1F808818802024151F2C800020401C36
:1010500080B27328FBD341F21110088044F6480097
:10106000108047F2480018802C8030BD202C0140B1
:10107000114944F648000880091D46F648000880DA
:10108000091D41F2111008800B48001F018841F032
:101090002001018009480021A0F86410A0F8621026
:1010A000A0F86010A0F85E10A0F85C10A0F85A102C
:1010B0000348418181827047182C0140980200202A
:1010C00060000020F0B54F4B4F480021DA7A0778D6
:1010D000802A27F001057DD31C684C4B02F01F02CB
:1010E00053F822204A4B14421A6802D042F02002E0
:1010F00001E022F02002474C1A60474E94F800C0ED
:10110000464CBCF1020FB4F9044043D1B3F808C017
:10111000CCF3C00ECCF3002CE6453BD03C4D2C3D2F
:1011200095F802C0BCF1000F04D0BCF1010F0FD044
:10113000A97033E05FEA025C30D55FEA826C2DD49F
:101140004FF0010C85F802C027F00405057025E07A
:101150005FEA025C22D45FEA826C1FD55FEA477CBB
:101160000BD447F004070770B0F802C0BCF1000FC1
:1011700006D0418027F0010707700227AF700DE00D
:101180004480002CF9DD47F001070770244FFF6A07
:101190004761F2E705704180318041811C4DC7886D
:1011A00095F846500FB9002C17DC077BAF4214D1DD
:1011B000B0F9027007F26667BC420EDC194FBF89B6
:1011C0005FEA477C09D45FEA877C06D45FEA427C09
:1011D00003D500E012E0FF0709D007785FEAC77C7B
:1011E00005D027F001070770418031804181C4801C
:1011F0000573500960F3CB221A60F0BD0570418081
:101200004181F0BDD00500201C090020D48F0008CA
:1012100098020020F306002018010020CA050020D3
:1012200060000020280A00202DE9F04796B0002435
:101230000C940D940E940F9472B69048816941F409
:1012400000718161816941F4806181614FF40040E6
:1012500002F0FCFD8A4D00212846FFF733FB0021F8
:101260002846FFF725FB874E00213046FFF720FB7D
:10127000854F0021384600F097F901204FF4704166
:10128000401C8842FCD32846FFF738FCB146304664
:10129000FFF734FC384600F093F94FF46020CDE9B5
:1012A00012048DF8454001204FF004088DF84400E9
:1012B00010948DF8508010A92846FFF7B1FC012347
:1012C0001A4605212846FFF7FCFC012302220621CD
:1012D0002846FFF7F6FC0123032207212846FFF7E3
:1012E000F0FC012304220F212846FFF7EAFC3846D0
:1012F00000F066F9684600F00EFA6148634E4C3023
:101300000090CDF80C80CDE901648020CDE9044047
:101310004000069080000790202008904FF4405035
:10132000CDE909046946384600F0D8F9012128467C
:10133000FFF7C8FA0121384600F036F901212846A6
:10134000FFF7B6FA47F2305115941598401C1590E6
:101350008842FAD301212846FFF7F2FCADF82C4071
:10136000A04640F2DC5A4FF4007420E05046CDF81D
:1013700054801599491C15918142FAD330880D99F2
:1013800008440D9070880E9908440E90B0880F990B
:1013900008440F90F0880C9908440C9001212846CD
:1013A000FFF7CEFCBDF82C00401CADF82C00BDF8BA
:1013B0002C00A042DAD30D98354A40F3CF163348BB
:1013C0000A3006830E9941F3CF1444830F9941F3F9
:1013D000CF1383830C9941F3CF1CA0F804C0ACF564
:1013E000C05C40F2C371ACF59B7C8C450ED2A6F577
:1013F000C856363E8E4209D2A4F5C854363C8C42BB
:1014000004D2A3F5C853363B8B4203D3D18841F4B1
:101410008041D180D188490407D41E49028B21F82C
:101420005C2F428B4A80808B888000212846FFF702
:1014300049FA0021384600F0B7F800212846FFF7A6
:1014400037FA00214C464846FFF732FA0220C10223
:10145000401C8842FCD32846FFF750FB2046FFF78C
:101460004DFB384600F0ACF8FFF736FA0A493C204D
:10147000087062B616B0BDE8F087000000100240A8
:101480000024014000280140080002401605002009
:10149000280A0020880C0020F0060020F0B5284B18
:1014A00040F22D4643F6FB255C6C264BB4F5FA5F03
:1014B00013DDB4F5FA4F10DC41F6AD17A4F5FA547C
:1014C000674306EBA7364FF4B5777C4305EBA414CE
:1014D00075106410C3E9045401E0C3E904651D6993
:1014E000D5605C69401A546110609168884202DAE4
:1014F0004942884200DC116010684443107E044178
:10150000906A21189162506A814200DD9062916A6E
:10151000106A814201DB084600E090629861116820
:101520004D43117C0D4108412918B2F91C00884235
:1015300004DBB2F91A00884200DC08B2F0BD0000FA
:101540003C0100201C01002010B54FF4005420463F
:1015500000F0ACF8002813D00A49087840F00800E1
:101560000870204600F014F80021074800F01CF82D
:101570000648C17E012903D10021C17601210177EE
:1015800010BD00006A060020440002402C0B002021
:10159000C10002D50249086070470249486070479F
:1015A00004040240000002400029016802D041F01A
:1015B000010102E04FF6FE72114001607047000029
:1015C00001684FF6FE721140016000210160416028
:1015D0008160C1603149314A0839904203D148687D
:1015E00040F00F0006E02D4A1432904204D14868C2
:1015F00040F0F00048607047284A2832904203D1FA
:10160000486840F47060F5E7244A3C32904203D1C8
:10161000486840F47040EDE7204A5032904203D1D0
:10162000486840F47020E5E71C4A6432904203D1D8
:10163000486840F47000DDE7184A7832904203D1E0
:10164000486840F07060D5E7154A111F904203D1F9
:10165000086840F00F0006E0114A1432904204D1AD
:10166000086840F0F000086070470D4A2832904248
:1016700003D1086840F47060F5E7094A3C329042B3
:1016800003D1086840F47040EDE7054A50329042BB
:10169000EAD1086840F47020E5E700000800024045
:1016A00008040240406880B27047000001460020F4
:1016B000CA0001D5034A00E0034A12680A4200D07A
:1016C000012070470004024000000240002A026826
:1016D00001D00A4300E08A430260704730B50368D6
:1016E00047F6F07293430C6A8A682243D1E90445B5
:1016F0002C4322438C692243CC6922434C6A224307
:101700008C6A22431A430260CA6842600A68826097
:101710004968C16030BD0021016041608160C160E5
:10172000016141618161C161016241628162704711
:1017300010B5114C8CB000212046FFF735FF204634
:10174000FFF73EFF0D4800900D480021CDE9010153
:101750006420CDE903018020CDE9050107910891BE
:1017600009910A9169462046FFF7B8FF01212046FA
:10177000FFF71AFF0CB010BD5800024004380140BA
:101780008807002010B501218CB0084602F068FBE4
:101790001E4C00212046FFF707FF2046FFF710FFF1
:1017A0001B4800901B48019000211020CDE9020148
:1017B0008020CDE9041006910791089109910A91C2
:1017C00069462046FFF78AFF012202212046FFF7E3
:1017D0007DFF01218DF82F1004208DF82D008DF84C
:1017E0002E100E208DF82C000BA802F025F80F20EB
:1017F0008DF82C000BA802F01FF801212046FFF7FE
:10180000D3FEFFF795FF0CB010BD0000440002406E
:10181000043801402407002030B540F6AA21204AB0
:10182000C184838B1488E31A9BB20F2B10D31288C8
:101830008283037E002253B11A4BB3F90A30062B80
:1018400005DB194B1B78022B03D0002B00D18284BF
:1018500030BD164B40F68B255B6CA3F22D14AC42C9
:101860000FD2428B521C92B24283642AF0D364227C
:101870004283B0F924208A4201DA02EB21118184EB
:1018800030BD41F29414A342FADBB0F92430002BAE
:1018900002DDA3EB211100E000218184428330BDF1
:1018A000FC06002060000020F30600203C01002020
:1018B00010B50446B0F9020043F69911484381136C
:1018C000E06840F26662504301EBA030E060B4F99A
:1018D000001043F6991251438A13216940F266635E
:1018E000594302EBA131216104F032FD6061A1880E
:1018F00040F6AB2208444010A0F515415539E0628E
:10190000914205D9A0F5F851FF39521C91421DD2E0
:1019100049F25451884202DDA0F5204002E0A0F5D2
:10192000F850FF38206300EB400040F34F00208563
:10193000B4F924104A42904201DA104602E088428B
:1019400000DD0846E083228461848AE0A0F5FE423F
:10195000FF3A41F255518A4214D8A2F6AA202063D8
:1019600000EB400040F34F002085B4F924205142A1
:10197000E183884201DA084602E0904200DD104629
:10198000404250E0A0F5D442AA3A8A4215D2A2F6CB
:10199000AA20206300EB400040F34F012185B4F9F9
:1019A00024004242E2832084914201DA104602E0A0
:1019B000814200DC0846608453E0A0F5AA42543A14
:1019C00041F256539A4215D2A2F6AB20206300EBA7
:1019D000400040F34F002085B4F924104A42904261
:1019E00001DA104602E0884200DD08464042E0830A
:1019F000218419E0A0F5804241F254539A4215D255
:101A0000A2F6AA20206300EB400040F34F0121859D
:101A1000B4F92400E0834242914201DA104602E028
:101A2000814200DC0846208462841AE0A0F5285236
:101A3000AB3A8A4215D2A2F6AA20206300EB4000FE
:101A400040F34F012185B4F92400E083424222840F
:101A5000914201DA104602E0814200DC0846404231
:101A6000A9E7B4F91E00A0EB40208013E080B4F990
:101A70002000A0EB402080132081B4F92200A0EBCD
:101A800040208013608110BD0121017670477047AE
:101A90001548164A4FF480410078042821D002F1FD
:101AA0003C03D08A9B88C01A00B22F2801DD0011A8
:101AB00008E0002801DD002007E00D4B984201DA24
:101AC000184602E0402800DD40209389184400B207
:101AD000884203DC40F26661884200DA0846908161
:101AE0007047918170470000F3060020B804002081
:101AF000C0FEFFFF38B54B484B4902880B889A1A45
:101B000092B20F2A71D30988484C01804FF0FF012F
:101B1000E2884FF47A7355044FF4967002D516227A
:101B2000009103E0950403D515220091014670E071
:101B3000D50402D514220091F8E7150502D5132229
:101B40000091F3E7550502D512220091EEE79505C5
:101B500002D511220091E9E7D50502D510220091A6
:101B6000E4E7150602D50F220091DFE7550602D5FE
:101B70000E220091DAE7950602D50D220091D5E7F5
:101B8000D50602D50C220091D0E7150702D50B220D
:101B90000091CBE7550702D50A220091C6E79507C9
:101BA00002D509220091C1E7D20702D00822009194
:101BB000BCE72289550702D507220091B6E79507B1
:101BC00002D506220091B1E7D20702D0052200918A
:101BD000ACE7A27AD20702D004220091A6E7A2893C
:101BE000D40603D503220091A0E719E0140702D51B
:101BF000022200919AE7540703D4940701D4D20734
:101C000002D00122009191E70020034602460146DE
:101C1000009002F073FEBDE838400248FFF748B973
:101C200038BD00001C0A0020FC060020280A002005
:101C3000F0B55948594982880B889A1A92B29C2A61
:101C400064D30988818056490A880146002A0B78A6
:101C500043F0020156D11646524A1C071568024647
:101C6000127822F0020274D54F4C0746E4887F7840
:101C70005FEA845C02D547F0010701E027F0010725
:101C80004770A704477802D547F0020701E027F024
:101C900002074770670401D4E70703D0477847F08D
:101CA00008074770640603D5447844F0040404E050
:101CB0001C0603D4447824F004044470EC0450D48B
:101CC000354C9A07247824F0100423D4324D4278FE
:101CD0002F7A2D78012A45F0100514D0022A16D04B
:101CE0002D4C042AA47804F1010C0CF0FF0C13D045
:101CF000072A25D0032A23D0052A21D0062A1FD05F
:101D000021F0100142E0B90702E00570F0BD39078B
:101D10000029FADB0470F0BDFA0601D41A060AD5D0
:101D20000170022C04D280F802C0BCF1020FF2D381
:101D300041F080012AE021F0100101708670F0BDB1
:101D4000877A7F06F7D5032C04D8017080F802C08B
:101D5000F0BD0FE05107D8D51906D6D443F0800165
:101D600014E002704178CB0701D18907F0D522F049
:101D700010010BE0E9040BD49907E9D4818AC82942
:101D800002D2491C8182E3E743F00A010170DFE7D8
:101D900002708682DCE70000D4060020FC060020EA
:101DA000FE06002098020020280A0020094944F677
:101DB00048000880091D46F648000880091D41F6C4
:101DC000CC4008800348001F018841F020010180B9
:101DD00070470000182C0140084946F6680008804A
:101DE000091D0880091D41F2555008800348001F55
:101DF000018841F02001018070470000182C01404B
:101E000010B5C28800210AB1032206E002890AB196
:101E1000022202E0428912B10122027000E0017048
:101E200004784FF4804344F6206244B1012C06D07C
:101E3000022C07D0032C01D14180818010BD43804A
:101E4000828010BD41F23331418040F6B731F4E772
:101E500030B5B1F86A5000231A240D22854202DC05
:101E6000B1F9680030BD4D88854202DBB1F9000050
:101E700030BD01EB82056D88854201DD144601E02D
:101E800013DA134604EB03024FEA52029A42F0D1EE
:101E900001EB830231F8231054889288521A001BF8
:101EA000424301EB622000B230BD31F9220030BD67
:101EB000054920B1086940F0800008617047034877
:101EC000486003484860704700200240230167458E
:101ED000AB89EFCD06494FF47A70CA68D20705D0B6
:101EE000401E0004000CF8D1FF207047002070470E
:101EF000002002400E4A0320A2F14C0182F83E006D
:101F0000002048810B490886C862C8830884488439
:101F100090620948816CB1F5206F01DBA3219162C9
:101F2000807A002802D0906A404290627047000098
:101F300060000020200500203C0100200449002012
:101F400048810881C862886202498862704700003F
:101F50006000002098080020F0B53B4988894A8934
:101F6000801A80B20F2866D388894881CA89374889
:101F70000B3A272A26D28A7822BB8268364B42F453
:101F800080728260324A354C354D12785607314A9C
:101F90000AD4344E36881680334A12881A80334A5F
:101FA00012882280324A09E0324E36881680324A40
:101FB00012881A80314A12882280314A12882A8077
:101FC00001228A702F4B304D19469A7F0968802A6A
:101FD00032D302F01F0255F8222011422CD0826821
:101FE00022F48012184E8260123614461215B77809
:101FF000521C62F38617254AB77093F816C01778FB
:10200000BCF1800F27F0020608D30CF01F0C55F826
:102010002CC011EA0C0F01D147F0020616701A7E8F
:10202000802A0DD302F01F0255F82220114207D159
:1020300044F400218160F0BD826842F48012D1E74F
:1020400024F40021F6E70000F006002098020020AA
:102050003C010020B0040020B2040020B4040020A1
:10206000B6040020A0040020A2040020A404002044
:10207000A6040020A8040020AA040020AC0400202C
:10208000AE040020D0050020D48F0008B804002042
:1020900070B5204881890289891A89B20F292FD306
:1020A000818901811C4B1D4819465D7A06681C4CCC
:1020B000096846F00402802D07D305F01F0554F887
:1020C0002550294201D126F0040202609A7B802A21
:1020D00017D302F01F0254F82220114211D10268D6
:1020E00022F002020260DA7A802A0ED302F01F0286
:1020F00054F82220114208D1016821F00801016042
:1021000070BD026842F00202ECE7016841F008018C
:10211000F5E70000F0060020D0050020980200201E
:10212000D48F0008F0B51D4C1B4A4FF0010C94F8F9
:102130003B5094F80AE0144692F83C3094F838404A
:102140002B43651CEEB2154D95F83D700025BEF190
:10215000FF0F0AD0BEF1000F06D18B4213D155708C
:102160000C2C01D282F83860F0BD834202D182F893
:1021700001C0F5E78B42F7D15570B80709E000BF01
:1021800082F83850F0BD8342FCD1F84382F801C098
:1021900080070028F4D0F0BD400400203C0100205E
:1021A000F0B5CA78002502F00F03D20601D58A786F
:1021B00013430A784FF00F0E12F0FF0F4FF0010299
:1021C0001CD004680F8802FA05F63740B74211D1D7
:1021D0004FEA850C0EFA0CF724EA070703FA0CF411
:1021E0003C43CF78282F02D0482F02D002E046612E
:1021F00000E006616D1C082DE4D304600C88FF2C00
:102200001ED944685FF0000606F1080702FA07F5D8
:102210000F882F40AF420FD14FEA860C0EFA0CF711
:10222000BC4303FA0CF73C43CF78282F00D145611B
:10223000CF78482F00D10561761C082EE4D3446086
:10224000F0BD0000F0B5144C002801DAE36900E0AD
:102250006368420D120185B2C0F301579540C0F387
:102260000346032F05D0C2020AD50322B24093438E
:1022700007E023F07062636823F07063636002E03C
:10228000AB4343F0706201B12A43002801DAE261F6
:10229000F0BD6260F0BD0000000001400246002079
:1022A00092680A4200D00120704741617047016185
:1022B00070470AB101617047416170470F4A104B86
:1022C00092F838105B5C834201D1012004E00D4B91
:1022D0005B5C834203D1002082F83A0070470A4BCE
:1022E0005B5C834201D18120F6E7084B595C814257
:1022F00001D18020F0E70320EEE700003C01002040
:1023000094930008A69300089A930008AC930008E1
:102310000A4810B501784FF000024C0708494FF009
:10232000FF0389684FEA017105D5002901DA82723D
:1023300010BD837210BD0029FBDBF8E73C010020D3
:1023400098020020F0B5194E194C0022E31CA6F1AA
:10235000060CB75CA518ED78FF5C0D430F43BD423A
:102360001FD01CF80270FF5C0F43BD4219D0154608
:102370000023A618F6780E43C6545B1C1CF80220F6
:10238000DBB2062BF5D3C17881700179C1700021D1
:102390004218491C15711CF80550C9B20629F7D31B
:1023A000F0BD521CD2B2032AD3D3F0BD668B000815
:1023B0004004002010B502460021064B06205C18A0
:1023C0006478944200D10846491CC9B20629F6D364
:1023D00010BD00003C010020214810B590F86710A6
:1023E00000222048012936D11F49898899BB1F49FD
:1023F0001E4B4C6C40F6B831B3F86E308C4227DD82
:102400001B49097821BB90F82711491CC9B280F8F3
:102410002711C8291CD380F827210146D0F82C4168
:1024200091F82811A34203DD052908D2491C01E0D7
:1024300041B1491E80F82811C9B2052902D30121F2
:1024400080F82611191B074C2C3C6162C0F82C3116
:10245000B3F5FA6F03D280F8262180F8282110BD49
:10246000880C002098020020CA0500203C010020B2
:10247000F30600204FF4C042C260002181620E22A8
:10248000028241F262024261082202834FF46042FA
:10249000428381834FF07842C0E9082140F6C4119D
:1024A00001807047B0F90010B0F90220891A41602C
:1024B0004269037E4A431A41836A13448362426A33
:1024C000934200DD8262836A026A934200DA82628A
:1024D000C268836A4A43017C0A410B41D118B0F9B2
:1024E0001C208A4201DA10467047B0F91A0088426F
:1024F000FADC08B27047000010B514481449B0F86F
:102500008C200B889A1A92B2B2F5437F1DD90988A4
:10251000A0F88C10B0F88A1020F8581F00224286CC
:102520000C480D4CC2888280C180C3898381248974
:10253000891AA4B2C4818160E11A0161074A818AC3
:10254000C182928A8282511A816110BD3C010020B1
:10255000FC060020500C0020200500206000002018
:1025600009480A49B0F8AA200B889A1A92B241F693
:1025700084639A4206D3098820F8AA1F4188818083
:1025800000214180704700003C010020FC06002033
:102590000D480178C90702D00C49098801E04FF6BF
:1025A000FA71C165094901201039088007482438AB
:1025B000018841F00101018004481838018821F0A8
:1025C00018010180704700003C01002024040040F5
:1025D0000A49D1F8902012B1521EC1F8902031F86A
:1025E0008A2F521C21F81A294A6A521C4A628A8F81
:1025F000521C8A8701F8380C704700003C0100200B
:102600001CB52D4890F83B3090F83C20934252D0B6
:1026100000248DF8044053408DF800309DF80030C0
:102620000122012B08D09DF80030022B09D09DF823
:102630000030042B0AD00DE01F498DF804204431EE
:1026400008E01D498DF80420463103E01A498DF851
:10265000042048319DF80420012A2CD190F83D3007
:102660009DF80040154AA34217D090F83E309DF8DF
:102670000040234208D0B0F84C30A0F84A300B8814
:102680001488E31AA0F84C3090F838302BB1B0F829
:1026900040301488E31AA0F8423012880A80A0F86B
:1026A000402010F83E1F9DF80020114300F801194A
:1026B0009DF8001001701CBD40040020FC060020A5
:1026C00070B5344D40212846FFF7E8FD8400802195
:1026D0002846FFF7E3FD44EA4004A9152846FFF722
:1026E000DDFD0443E1B22C4C94F870508D4250D083
:1026F0004D4084F87010012D03D0022D01D0042D1F
:1027000047D194F87400A84384F8740094F87320B7
:10271000AA420FD084F8735094F8722001238B40A2
:102720001A4207D11A4384F8722094F87110491C98
:1027300084F8711094F87110042928D330B101285D
:1027400011D002280FD004280DD012E01348C18800
:1027500021F04001C1802078002184F83B1020F056
:102760006000207005E0217841F02001217084F89C
:102770003B000B4994F83B0091F82720904204D08D
:1027800081F8270007492020087000F00DF884F830
:102790004C5070BD001001403C010020280A002070
:1027A000880C0020F006002070B50D4D4021284611
:1027B000FFF774FD840080212846FFF76FFD44EA8F
:1027C0004004A9152846FFF769FD04430548072181
:1027D00000F8704F0171002141708170C17070BDAF
:1027E000001001403C01002070B5344890F83A10C8
:1027F000CA43920761D001F0030280F8392090F8B3
:102800003D305B061B0E80F83D30012A01D0812A45
:1028100002D15B1C80F83D300278D2074DD0DBB28C
:1028200003F00102C3F34004A24246D1B0F84E4087
:102830000025641CA0F84E40204CA0F8505090F8A1
:102840003E60A47AB24202D080F83E200DE0A60796
:10285000B6EB837F02D080F83F5006E090F83F301F
:10286000642B02D25B1C80F83F3090F84030642B20
:102870000CD25B1CDBB280F84030022B06D204F095
:102880000103934202D1022280F84020012901D0A5
:10289000002912D190F83820C16D00EB82029161BD
:1028A0000163D0E906121144D0E908231A44114407
:1028B000826A1144C26A1144416370BD3C01002028
:1028C000FEE700002DE9F04F00BF00209E4E9F4A1A
:1028D000A6F51271A6F5BE79A6F1440B06F1440ED9
:1028E000804601F5E074A1F1780301F5457A1D5C9D
:1028F00015F0C00706D0402F51D0C02F77D0802FC1
:1029000076D004E115F01F0504D0154440F080078F
:102910002F7201E082F80880012826D0022824D0F6
:10292000032822D0042820D008281ED010281CD02C
:10293000874D55F820C0DCF8005054F820703D4019
:10294000CCF80050824D55F820C0DCF8005056F805
:1029500020703D43CCF800501D5CAD0659F8205066
:102960002F6813D53AF810C03EE051F820502F6878
:1029700054F820C007EA0C072F6051F820502F6848
:1029800056F820C047EA0C072F60E5E7DFF8B8C12A
:102990000CF1F00C5CF820C007EA0C077EE015F0A3
:1029A0001F0504D0154440F080072F7201E082F823
:1029B000088001281DD002281BD0032819D0042824
:1029C00017D0082815D0102813D0614D55F8205085
:1029D0002F6854F820C007EA0C072F605C4D55F8AB
:1029E00020502F685BF820C047EA0C0756E00BE048
:1029F00056E051F820502F6854F820C007EA0C0721
:102A00002F6051F82050ECE715F01F0505D0154454
:102A100040F0800785F8217001E082F821800128CC
:102A200025D0022823D0032821D004281FD008282D
:102A30001DD010281BD0464D55F820C0DCF80050A2
:102A400054F820703D40CCF80050414D55F820C05E
:102A5000DCF800505EF820703D43CCF800501D5C5F
:102A6000AD0615D53A4D3AF81070CC3514E051F852
:102A700020502F6854F820C007EA0C072F6051F847
:102A800020502F685EF820C047EA0C072F60E6E769
:102A90002D4D3AF81070E03D55F820502F6036E08B
:102AA00015F01F0505D0154440F0800785F821700A
:102AB00001E082F82180012830D002282ED003289E
:102AC0002CD004282AD0082828D0102826D0204D21
:102AD00055F820C0DCF8005054F820703D40CCF888
:102AE00000501B4D55F820C0DCF80050164F8837B9
:102AF00057F820703D43CCF800501D5CAD06B1D4B2
:102B0000114F3AF81050E03F57F820703D60401CDC
:102B1000C0B21128FFF4EBAEBDE8F08F51F82050A1
:102B20002F6854F820C007EA0C072F6051F8205096
:102B30002F68DFF814C00CF1880C5CF820C047EA5D
:102B40000C072F60D9E7000060920008D005002034
:102B50005C9000084FF40771C1824FF45861018303
:102B600040F6145181837047F0B5C48AB0F9006013
:102B70008681B0F90250C581B0F9043002270021E6
:102B800001220382AB4204DBB54202DDC7804281F1
:102B90000CE0B34204DBAE4202DDC78041811CE0A1
:102BA0009D4205DBB34203DDC2804781018115E010
:102BB000B54204DB9E4202DDC280418105E0AE42A7
:102BC00005DB9D4203DDC1804281078106E09E4214
:102BD00004DBAB4202DDC18047810281C3884589A5
:102BE00000EB430700EB4505BB89AE899B1B0FFA41
:102BF00083FEA0F812E00689AB8900EB460CBCF816
:102C00000CC0A3EB0C038382B0F91830B7F90CC0E9
:102C1000A3EB0C0CB4EB4C0F04DA80F82010A3F1FA
:102C2000A10113E0A64503DD80F82010B9890BE06F
:102C300026B1012E04D0022E10D004E0062100E0BF
:102C4000052180F82010A989091B6D31418309B243
:102C5000B1F5586F04DB5B1E438304E00421F0E709
:102C6000002900DC4283418B8183F0BD0B490022A7
:102C700088760A62CA614A62094A32F9103002EB68
:102C800040028B62B2F90220CA62064A32F8100092
:102C90000882A1F86000A1F862007047EC010020F2
:102CA000BE930008B29300082DE9F05FF748F84999
:102CB00082880B889A1A92B20F2A44D30988F54A5F
:102CC0008180814611880124F348F44E002579B3B0
:102CD000491E1180C573F24A85620168B2F902206B
:102CE0004F0742F6AA2318D4F78847F40057F78015
:102CF000EB4E3678B60709D5866826F080068660E2
:102D0000A0F87C5080F87E5080F87F50CE0404D428
:102D100080F8F040C0F8EC5003E080F8F0504E0727
:102D200007D49A4205DB80F8F440A0F8F25004E0A2
:102D300010E080F8F4504E0703D49A4201DBC90733
:102D400003D080F81151BDE8F09F80F81141A0F840
:102D50001251F8E78046B0F8181143F698208142E6
:102D600002D2491CA8F8181101F0DEFDCD4FDFF8A2
:102D70001CB397F85000ABF1180B10B1FEF7A2F995
:102D800005E09BF8001021F001018BF80010FFF71F
:102D900023FB00F0CBF9C44841F26801426C4FF4C8
:102DA00000608A4201DBC14904E0B2F57A6F02DAC1
:102DB000BE49091D086097F85100DFF8DCA2C10781
:102DC000BB48BC4FAAF12C0A3AD0817B802933D36F
:102DD00098F800309B072FD498F80F308AF8053008
:102DE000AF4B514693F800C02CF0020C83F800C0A2
:102DF000ABF80250CBF814509BF800C02CF0010C3B
:102E00008BF800C0B3795B0611D44B89B3F5FA7F18
:102E100003D25B1CAAF80A3012E040F63C708242F2
:102E200001DD002007E108208AF8034003E1CD70AE
:102E30000020AAF80A50FEE08AF80350AAF80A50C7
:102E4000D8F80830190501D50820F4E0954991F823
:102E50003FE05FEACE7149D0954898F80F208AF894
:102E60000520407A414680284CD30878400735D465
:102E7000F088800405D500BF23F02000C8F80800C2
:102E800034E0ABF80250CBF814509BF800C043F08C
:102E900020002CF0010C8BF800C088608448C37DB2
:102EA000802B0AD303F07F0C00684FF0004323FA15
:102EB0000CF3184201D10C7100E00D710879C007C4
:102EC00002D15FEA8E7005D50320032A01D08AF86B
:102ED0000840B0E00020C8F82850ACE023F0200003
:102EE000C8F80800F08820F40050F08098F8260117
:102EF000444601280BD06B4890F8630048B1FDF7B9
:102F0000A1FF0FE0086840F004000860B4E7092062
:102F100091E0A068C10502D520F0080001E040F072
:102F20000800A06094F8462002B343F69911012AE4
:102F300023D043F6FE70032A26D03A78C2F38102EA
:102F4000012A02D0022A00D0801CA4F814015A4899
:102F500090F85E00042814D04FF48040A4F8440098
:102F6000504890F87000012811D01FE043F21E5025
:102F7000A4F8140143F23330F0E742F6CC40A4F851
:102F80001401A4F84410EBE7A4F81401E6E738783C
:102F900042F26661C0F38100012810D0022811D0EE
:102FA00041F6E120A4F81401A4F84410FEF78AF8D1
:102FB0009BF80010C90708D0BBF8021007E0A4F87E
:102FC0001411F1E74FF40050ECE735488188A9F877
:102FD000121008B2B4F944104FF480424843C0F3D1
:102FE0008F315046AAF81210914200D942823349DB
:102FF0000978C90605D5428A41F233318A4200D2A6
:1030000041822189C1F3C002C1F300218A4205D166
:10301000428A40F6CC418A4200D94182B17AC9073E
:1030200000D04582BAF81200A06200287FF7F9AEFE
:1030300023480570022099F81A1099B9022841D046
:1030400080B119490B789C0608D5B479640605D57A
:103050001A4C2478E40964F386130B70F18821F488
:103060000A61F1801049496C4E290ADBF1880B0690
:1030700007D521F08001F18009490B7823F0020384
:103080000B7089F81A0088F80F005CE634090020FC
:10309000FC060020FE06002098020020280A0020DE
:1030A000CA050020880C00203C010020100C0140C3
:1030B000D0050020B804002060000020D4060020C5
:1030C00010070020398F0029BBD143F6982139879A
:1030D000B7E770B500230C8863F30F02012505FAEA
:1030E00003F6344206D0C3F10F0605FA06F1114388
:1030F00061F30F025B1C102BF1DB028070BD70B519
:1031000000230C7863F30702012505FA03F6344225
:1031100006D0C3F1070605FA06F1114361F3070271
:103120005B1C082BF1DB027070BD0000F0B51F487E
:1031300090F866301E48012B816821F4006232D17C
:103140001C4BDE8874062ED41B4D0F054FF0000477
:10315000B5F902501ED4194A526C642A11DC40F6AB
:10316000386295420DDAB2040BD4027852070ED4BD
:10317000B0F8D42040F6B835AA4203D2521CA0F8C9
:10318000D420F0BD41F4006181605C81F0BDA0F805
:10319000D440F0BD41F2CD018D42FADD997AC907E4
:1031A000F7D18260F3E78260F0BD0000880C002058
:1031B00098020020280A0020CA0500203C010020B7
:1031C000F0B5364D364F044695F83B0097F83B1066
:1031D00023780843EE1C6278834205D1E0781146DB
:1031E000FEF7A0FF207908E094F802C084450CD1D6
:1031F000E1781046FEF796FFE07905F82F0F287862
:10320000805D6870287BE877F0BD82421DD1614601
:103210001846FEF787FF95F84E1095F83B0081425F
:1032200007D1B97A09B1A17900E0617985F82F1049
:103230001EE06978012901D0A17922E0617927E0B7
:10324000297841F00401297012E0E1788142DBD154
:1032500019466046FEF766FF95F84E1095F83B005C
:1032600081420AD1B97A09B1617ADFE7217ADDE7D3
:1032700015F82F1F895D6970C5E76978012906D0A7
:10328000617A85F82F10B97A0029F1D1D8E7217A2F
:1032900085F82F10B97A0029EAD0D1E74004002040
:1032A0003C0100200B48017821F0020100F8381B96
:1032B000002100F8181941778177332181854185F4
:1032C00008214184012100F81F1C034880F83910AF
:1032D00070470000400400203C0100200D4900B56B
:1032E0000B4851F8012F40F8032F89888180084846
:1032F00001210930FFF726F8054802211330FFF7B6
:1033000021F8034804211D305DF804EBFFF71AB8DB
:10331000400400203C010020094944F64800088090
:10332000091D46F648000880091D41F21110088069
:103330000348001F018841F0200101807047000010
:10334000182C01402DE9F047664C674B0025A0780A
:103350000126654A103305287ED2DFE800F003130A
:10336000113E1100108820F0010010801D805F4880
:103370000580001F0580001F0580FFF7CDFFA670A8
:10338000BDE8F087594941F244401C39088057494B
:1033900045F6580024390880091D47F25800088076
:1033A00052492020283908800020401CC0B27328D0
:1033B000FBD3FFF7B1FF4C4984F85C502C3147F642
:1033C000906008804848143006801D80108840F0C6
:1033D000010010800220A070D2E700215FF0010000
:1033E00004EB410204EB4003B2F85020B3F8503034
:1033F0009A4200D20146401CC0B20628F0D33C4895
:10340000405C84F83900FFF74DFF1D2000F0F3F910
:1034100000F076F8374E38484FF4807996F83B1034
:10342000012904D002291BD0042930D047E04021D3
:103430008046FEF733FF870080214046FEF72EFFCF
:1034400047EA400749464046FEF728FF074347F052
:10345000010084F83B0000E03DE0224809302CE008
:1034600040218046FEF71AFF870080214046FEF784
:1034700015FF47EA400749464046FEF70FFF07435E
:1034800047F0020084F83B001648133015E0402155
:103490008046FEF703FF870080214046FEF7FEFED0
:1034A00047EA400749464046FEF7F8FE074347F023
:1034B000040084F83B000B481D3002F033FE94F802
:1034C0002F0086F838001D2000F0ABF90420A07012
:1034D0000A48057054E7108820F0010010801D8014
:1034E000A5704DE740040020000800403C2C01403E
:1034F0006C8B00083C01002000100140F306002006
:103500002DE9F041344C14F82F0F344DE072402176
:103510002846FEF7C3FE860080212846FEF7BEFE41
:1035200046EA4006AF1539462846FEF7B7FE064381
:10353000207BF1B22F3C814215D084F83C00402121
:103540002846FEF7ABFE860080212846FEF7A6FE41
:1035500046EA400639462846FEF7A0FE064384F8B0
:103560003B60FFF74DF81E4D95F83B00012827D032
:10357000022828D0042829D0174894F83B10273077
:10358000085C04F8300F14F80109FEF713FF04F883
:103590002F09A87A00B10120607001F05DFA94F85B
:1035A0004E0094F83B10884206D094F83800062864
:1035B00002D2401C84F8380084F84E10BDE8F08137
:1035C0000548093004E00448133001E002481D308A
:1035D000BDE8F041FFF7F4BD4004002000100140B9
:1035E0003C0100202DE9F041524991F87200AA28CF
:1035F0007ED191F8730055287AD14F4C00200A5C97
:103600002254401CC0B27428F9D34C4E2069C6F82D
:103610000100A08AA6F80500D4F81600F060D4F8DE
:103620001A003061D4F81E001234706102F020FDDF
:103630004349608A888102F035FD207D123CC00735
:10364000307802D040F0040001E020F004003D4951
:1036500030704FF480403C4D886114F8280F85F895
:103660002000608B6880A08BA880E08BE880208C95
:103670002881608C354F688194F8240087F8D20047
:1036800014F8011C304686F83B100026C0F8946000
:10369000FFF724FE2E48A18E0183E18E4183218F06
:1036A000818394F84210283C012908D0022901D0D6
:1036B000032909D0297821F00C01083107E0297885
:1036C00021F00C01091D02E0297841F00C0129705C
:1036D00094F86E20012162B1012A01D0022A0BD098
:1036E00087F8461094F864301A4A4BB1518108E0CB
:1036F00014E087F84660F5E7022287F84620F1E7F4
:10370000568194F8701001290AD094F86D1051B1C7
:1037100001290BD04FF48051A0F87610BDE8F0815C
:1037200044F21C71F8E74FF40051F5E741F25551AE
:10373000F2E7000000FC0008880C00203C0100209B
:1037400060000020200C0020B80400209802002017
:1037500020050020280A00207CB50121082000F067
:10376000A3FB4FF48070ADF8040010248DF80740DF
:1037700001208DF8060001A91548FEF711FD012171
:10378000092000F091FB01211248FEF75BFD0820A3
:10379000ADF8000004208DF803000F4E03258DF8CE
:1037A000025069463046FEF7FBFC08213046FEF722
:1037B0007CFDADF800408DF803408DF8025069465D
:1037C0003046FEF7EDFC10213046FEF76EFD7CBD65
:1037D0000014014000023000000C0140FEE7704779
:1037E00000F01F02012191404009800000F1E0201B
:1037F000C0F88011704700F01F020121914040097C
:10380000800000F1E020C0F88011704700F01F0236
:10381000012191404009800000F1E020C0F8001132
:10382000704700F01F02012191404009800000F123
:10383000E020C0F80011704770B50F23C4780178FC
:103840000122F4B1144C2468457804F4E064C4F512
:10385000E064240AC4F10406E3408478B5401C40C7
:103860002C4301F1E021230181F80034007800F0BD
:103870001F018A404009800000F1E020C0F80021CB
:1038800070BD01F01F0082404809800000F1E02077
:10389000C0F8802170BD00000CED00E00249084333
:1038A00002490860704700000000FA050CED00E0D6
:1038B0002DE9F05F00261D20FFF792FF6C4CDFF82A
:1038C000B4B1A4F1B000A77E90F83810DFF8A8E1F9
:1038D000DFF8A8A100258F427ED0E776A176626A44
:1038E000036B5A434FEA12499BF80820120702D58E
:1038F0001EF8012000E00A4694F812C0BCF1010F46
:1039000009D004EB4206B6F902C0C4F828C0B6F9E3
:103910000460E6620CE043F6FF7CC4E90A5C90F8C0
:103920003DC05FEACC7C01D012B102E0052A00D193
:10393000012600EB47074FF0804CBF893F04B7FBDF
:10394000F3F3E361476BBCFBF7F7276294F813C00E
:10395000BCF1000F06D0BCF1010F05D03B4403EBD6
:10396000D3735B10636201E03B466762DFF810C10E
:103970004FF6FF7707EA8307ACF808709AF80070F3
:1039800090F80A8090F83DC0082F08F003070CF06B
:10399000030C05D067450BD1B8F1000F05D008E046
:1039A000674505D0B8F1000F03D05B42636200E0C9
:1039B0006562C6B1636A002B03D006DD228D05E087
:1039C0000AE0304B33F8122000E0A28DA4F860200A
:1039D000227822F0200222709AF80020042A07D0D0
:1039E000082A05D012E0B4F8603003EB0902EDE7D5
:1039F00080F8405065629BF80800000701D51EF86A
:103A00000110204830F81100A4F860001E49606AD7
:103A100009883E314843B4F8601001EB204006B2FB
:103A20001D20FFF7F3FE606A002807D021784FEAD7
:103A300081600ADD002804DAA08D09E0B4F8600096
:103A400006E0E06AB04208DB0CE0002802DA208DD4
:103A5000208208E0A06AB04204DD208241F020000C
:103A6000207000E02682257565752586BDE8F09FEB
:103A7000EC01002098020020A0930008F30600202B
:103A8000000A0020B29300082404004043184FF4B9
:103A90008042934210DD904202DD104600210BE08F
:103AA000914202DD0020114606E08003B0FBF3F0F6
:103AB00000B2C0F5804109B241EA00407047F0B55C
:103AC00000224FF46A740E25C460826205824FF4AE
:103AD000834608274661078343F6FF7C4283A0F8AC
:103AE0001CC040F249234FEA8C3E8360C0E9082E97
:103AF000CC608A620D824E610F834A83A1F81CC09C
:103B00008B60C1E9082EF0BD002181620949C160C6
:103B10000E2101824FF6BF514161082101834FF40C
:103B20004041418343F6FF718183090701620249E5
:103B300041627047638A010000C0FF0F064941F6E9
:103B4000A260088005480168054A01F4E06111435C
:103B50000160BFF34F8FFEE7442C01400CED00E005
:103B60000400FA0538B501210D2000F09DF94FF44D
:103B7000E060ADF8000018248DF8034003258DF8AF
:103B8000025069460D48FEF70BFB4FF46040ADF85C
:103B900000008DF803400A4C8DF80250694620461B
:103BA000FEF7FEFAA014ADF8000048208DF80300DF
:103BB00069462046FEF7F4FA38BD000000080140CF
:103BC000000C0140F0B50121CE028DB0304600F06E
:103BD0006BF9594F384601F0B1FB08A801F0DAFD46
:103BE0004FF45860ADF824000024ADF820402020A8
:103BF000ADF82200ADF8264008A9384601F07CFD5A
:103C00000021384601F0CFFD4FF6FF71384601F034
:103C1000D4FD01220021384601F060FD0121384623
:103C200001F048FB04A801F060FBADF810607010D3
:103C3000ADF81200ADF81440A220ADF816007000E7
:103C4000ADF81800ADF81A40ADF81C4004A938468C
:103C500001F03AFB6025ADF80050ADF80440ADF836
:103C60000840ADF80C40ADF80240ADF80640ADF8A4
:103C70000A40ADF80E406946384601F01FFC69461F
:103C8000384601F061FC6946384601F0A7FCADF802
:103C900000500125ADF8045040F61450ADF8060070
:103CA000ADF80840ADF80C40ADF80250ADF80A4050
:103CB000ADF80E406946384601F0D4FC0121384683
:103CC00001F01CFB0821384601F038FC314638462B
:103CD00001F07AFC0821384601F0BEFC3146384636
:103CE00001F0F2FC7021384601F0FBFC18208DF841
:103CF0002C008DF82D408DF82E408DF82F500BA8FC
:103D0000FFF79AFD0C480C30018841F080010180DA
:103D100009481430018841F001010180001F04802E
:103D20000121384601F0F4FA8DF828500121384677
:103D300001F0F8FA0DB0F0BD002C01407047000012
:103D400070B50189C1EB411101EB4101CA0B428100
:103D50000B49104603F040FD09480C38B0F90C201F
:103D60000168B0F90E4001FB02F54368614303FBB3
:103D7000145503FB0211AD138913C0E9055170BD41
:103D80000C0A002040F21341416008218160862125
:103D9000C1604FF4804101614942416100210162EB
:103DA000C16270470162704710B501884288891A64
:103DB00009B20183B1F5005F02DBA1F5804104E0A7
:103DC00011F5005F02DC01F580410183B0F9182094
:103DD00041685143C1618368846A5343C2681B12BE
:103DE000624303EB2222036A1A44114402628A13DB
:103DF000426241698A4203DB01698A4200DC114662
:103E00008A1AC0E90A21028E4FF40373594302EB68
:103E1000A13202860B4A1278082A04D10A4A936F0B
:103E200003EBA1319167B0F93010B1F5804F02DD9D
:103E3000A1F5804103E0002902DA01F58041018605
:103E400010BD0000F30600203C0A0020034A516820
:103E500021F44041014351607047000000100240CE
:103E6000044A0029516901D0014300E081435161B6
:103E70007047000000100240044A0029D16901D0B7
:103E8000014300E08143D16170470000001002400F
:103E9000044A0029116901D0014300E08143116106
:103EA0007047000000100240044A0029916901D0C7
:103EB000014300E08143916170470000001002401F
:103EC000044A0029D16801D0014300E08143D16058
:103ED000704700000010024030B524494A6812F0D3
:103EE0000C03234A03D0042B01D0082B26D00260F8
:103EF0004A680F231F4C03EA1212A35C0268DA40DF
:103F000042604B68072505EA1323E35C22FA03F3BA
:103F100083604B6805EAD323E35CDA40C2604B68F8
:103F2000032403F4404104EA933303EB9161114B02
:103F30001B1F595CB2FBF1F1016130BD4A680E4BA9
:103F40001A404B68140103F4803303D5C2F3834253
:103F5000113202E0022404EB924213B14B689B033E
:103F600001D5064B00E0024B5A43C0E70010024067
:103F700000127A000400002000003C0800093D0007
:103F80002DE9F041274CA61540212046FEF786F981
:103F9000850080212046FEF781F945EA400531463B
:103FA0002046FEF77BF90543EDB240212046FEF79F
:103FB00075F9870080212046FEF770F947EA40072F
:103FC00031462046FEF76AF90743F8B2A842DBD132
:103FD00040212046FEF762F9870080212046FEF747
:103FE0005DF947EA400731462046FEF757F9074397
:103FF000F8B2A842C8D140212046FEF74FF9870009
:1040000080212046FEF74AF947EA4007314620461C
:10401000FEF744F90743F8B2A842B5D12846BDE8F7
:10402000F08100000010014010B50268416802FBF9
:1040300002F301FB01330D4CA34211D91B0E0E3BC1
:104040000B4C9BB212B234F8133009B25A435943A5
:1040500042F38F3241F38F31C0E90221012102E0A6
:10406000C0E902210021017410BD0000E10BBF0E68
:104070000C8800082DE9F05FF848F94902880B88A0
:104080009A1A92B20F2A7DD309880180F548024618
:104090008189D2884B0703D48B0701D4CB0702D088
:1040A00042F4007201E022F40072C28081460807E7
:1040B00002D44846C90604D5B9F8061041F00101FA
:1040C00002E0C18821F00101A9F80610E548FDF7DA
:1040D00097FEE548B0F93A10B1F5804F02DA491C75
:1040E000418703E0E0494FF480404887DF4E41F6C6
:1040F000CC41DF4CB06C884203DDA06820F010009A
:10410000A060DC49DFF870830025088828B1401ED4
:104110000880E57388F8005028E0B9F806004204EA
:104120001BD4B9F80C10CA0617D4090715D4010618
:1041300013D4810611D401050FD4410603D5CF490C
:104140000978090609D5410707D4C10505D4010737
:1041500003D4810401D4C00608D5C948E573C94910
:1041600088F80050C5830D8080F82A50E08FC6493A
:10417000DFF818E348B1401EE087087820F002001D
:10418000087000E09AE0E5730BE0087840F0020068
:10419000087098F80000012805D19EF80000062854
:1041A00001D188F8005098F80000DFF8C4A2DFF8C9
:1041B000E0B20127AAF12C0A0A2873D2DFE800F046
:1041C000F77E057EF6F57E72F4F3E07B09281AD0BF
:1041D000DFF8C09202287DD0B4F8400018B399F8F7
:1041E000680040F63A2201282BD0C4F8D85084F851
:1041F000EA50CAF82050B4F9301001F21D50904234
:104200002FD810232EE095484430FEF733F9FDF700
:1042100071FEDBF82C10A04841F39101CBF8281077
:1042200089038162FDE1BBF814202286DBF82C2093
:10423000CBF83420DBF82820CBF83020A4F84070ED
:1042400015E09648C4F8D80084F8EA70B4F9301044
:1042500001F21D53934201D8102300E020231022C5
:1042600002E020231022002000F054FB208699F861
:1042700068008B490128706C40F2DC524FF4927355
:1042800011D0904203DABBF90A209A4211DBB4F84C
:10429000403040F6C4125B1C9BB2A4F840309342FD
:1042A00007D20EE022E1904208DABBF90A009842F8
:1042B00004DA88F8005084F8EA504D83BDE8F09F96
:1042C00008E0694AD268002AF8DC42F6E0629042CF
:1042D000EFDAF3E7706CCAF828008AF80770714FBC
:1042E000A4F8405084F8EA50797F5646A1B1F87F8F
:1042F00090B3208DB4F9301000B20A23052200F0EB
:1043000009FB2086FD777D77B4F930104FF48040AB
:10431000814254DD2086D1E794F84610022903D16A
:1043200099F86D10022918D000B25F4901F066FCBF
:10433000A4F8E400B4F9E410A06A884200DB08465F
:1043400000B2B08299F84D104F460029B4F93010F0
:1043500007D03623052207E02DE0534900B2B031E3
:10436000E4E740F24713362200F0D4FA2086B4F98D
:104370001601B4F91411884208DA97F84D1011B1FA
:1043800000F102000CE000F1080009E010DD3179D5
:1043900001F10101C9B231710229B5D33571401E55
:1043A000A4F81601B0E72FE00DE052E04DE081E007
:1043B000A4F81611A8E740F266602086A4E7002959
:1043C00087DA25867AE73949D4F8DC00884202D2B8
:1043D000401CC4F8DC00E07B082803D1D4F8DC00E2
:1043E00088420DD388F80050A068C10502D520F09E
:1043F000080001E040F00800C4F8DC50A0605DE770
:10440000BDE8F05F02F044BCE07B092801D02586BE
:1044100049E1DAF81C005746401CCAF81C00022883
:1044200009DD388D012301B2388B052200B200F07E
:1044300071FAFD61B8620948398D44300180B6F8DF
:1044400044104180FEF72EF864E7BDE8F05F04F009
:104450009FB81748007809287ED02FE7340900203C
:10446000FC060020280A0020200500203C01002036
:104470009802002000070020F3060020D406002048
:10448000C80800201E000020CA050020F4060020F5
:1044900060000020880C00206808002034F3FFFF33
:1044A000A8090020500C0020FE890008C0D401009B
:1044B000540200209049914B0888401C82B29048D9
:1044C0000A80C82A04D390F800C0BCF1010F18D0AC
:1044D000B2F57A7F04D390F800C0BCF1020F10D07F
:1044E000B2F5FA6F02D30278032A0AD0E07B801E6D
:1044F000082872D2DFE800F00F9EDAEC04F866902C
:10450000DCE605700D80B9F8061021F40061A9F809
:1045100006101F70EAE7FDF7FBFE3078400611D564
:104520007848807804280DD0706C82280ADAB07A36
:1045300096F83D1000F0030001F00301884201D01D
:1045400001F05CFD98F80000062886D086F83F5000
:10455000B06C40F3110000E0A5E083036A4ACBF899
:104560002C00801093628103CBF828006748816299
:10457000FDF7C0FC8AF80770B4F81401A4F816011E
:10458000706CA4F88250B0F5437F08DD4FF4804092
:10459000A4F880007AE000BF88F800008EE64FF4AF
:1045A0008041A4F88010A16821F48061A16040F2EC
:1045B0008A21884204DA3078400601D402F054FAA5
:1045C000A0686BE0706CB0F5437F07DA9EF80010CE
:1045D000062903D08EF800507EE085E04C48017833
:1045E00021F040010170FDF785FC43F6FE70A4F850
:1045F0001601DC34FDF78CFE464810F8341F21F01C
:1046000001010170414925608D623F498D62082199
:1046100088F80010456451E63F48FDF72BFFFDF791
:1046200069FC716CCAF8281041F27C510920CAF863
:104630001810B1E799F80600C006AFD4706CB0F559
:104640007A7F30DDFDF764FE3078400611D52D48C5
:10465000807804280DD0706C82280ADAB07A96F837
:104660003D1000F0030001F00301884201D001F089
:10467000C5FC86F83F50B6F84800208601B24FF4DA
:104680008040814200DD2086FDF734FCA06840F4C4
:104690008060A06096F838100529BCD140F0100069
:1046A000A060022078E788F8005007E6706CB0F54B
:1046B000437F03DA9EF8001006298BD1B9F8061063
:1046C00021F02001A9F80610FDF722FE042063E77F
:1046D0009EF80000062802D088F80070EEE50F4929
:1046E00009200870052057E7064885708EF80050AD
:1046F0008BF85E5065E600001600002014000020D4
:1047000015000020400400209808002068080020C0
:10471000020700203C0A00207809002054020020F3
:1047200030B585B001210420FFF7BEFB4FF40040F7
:10473000ADF8100048208DF8130004A91848FDF7C3
:104740002FFD01210846FFF797FB40F68C20ADF8BE
:10475000040003240020ADF80040ADF80200ADF8DD
:1047600006004FF080456946284600F0C5FF1C2032
:104770008DF80C008DF80D408DF80E4001208DF85D
:104780000F0003A8FFF758F801221146284600F051
:104790008DFE0121284600F0BBFD05B030BD0000B4
:1047A00000080140704700002DE9F041304CE078EE
:1047B00000285AD12078002857D0401E10F0FF0062
:1047C000207052D14FF49670208272B6294F45F274
:1047D000AA50A7F872000020FDF76AFB264D1320AF
:1047E0002860FDF777FBA8BB3420E8600220286131
:1047F000224E6E61286940F040002861FDF76AFB97
:1048000040BB00211E4A08465FEA255312F800C04B
:10481000BCF1FF0F00D00121401C80B29842F5D3BB
:10482000C1B9C4E9067639260127A06910F8011B31
:1048300010F8012BA061E06901EB022102886A6196
:104840002F6120F8021BE061FDF744FB10B9761ED2
:10485000B6B2EAD20120FDF72BFB62B601F022FCD2
:104860000848816821F480418160BDE8F081000042
:10487000F0060020880C00200020024000FC000808
:1048800000FC0008980200201948016841F010015E
:104890000160016821F003010160016841F002013B
:1048A000016014484168416041684160416841F4D9
:1048B00080614160416821F47C11416041680E4A89
:1048C00011434160016841F0807101600168890114
:1048D000FCD5416821F003014160416841F00201CB
:1048E00041604168C1F381010229FAD1704700009B
:1048F00000200240001002400000280830B5044C9F
:10490000039D6080A180E2802381658130BD00002D
:104910001C0A00200A44824201DA10B27047C91A08
:104920008142FBDD08B270472DE9F0434348DFF8D0
:104930001081DFF81091C17F457A046801260023B9
:10494000414A424880292BD301F01F0158F8211019
:104950000C420146096802D041F4805101E021F483
:1049600080510160CF0417D48F0415D5977AFF07C3
:1049700007D0538199F800C02CF0020C89F800C0D0
:104980000AE090F84670BFB14FF0020C012F18D02A
:1049900080F8463080F81AC10F0B67F34D31016083
:1049A000802D2AD305F01F0158F821100C42016810
:1049B0000CD041F004010BE080F8466080F81A3119
:1049C000EAE780F846C080F81A61E5E721F00401C3
:1049D00001604C070DD44C050BD5947AE40708D040
:1049E000538199F8005025F0020589F80050C0F86D
:1049F00098308C0864F38A210160917AC90717D135
:104A0000134991F86410012912D11249496C3229D5
:104A10000CDC0178490709D50189090506D4D0F8CD
:104A2000981047F23054A14204D95681C0F898300A
:104A3000BDE8F083491CC0F89810F9E7D0050020C4
:104A4000D48F0008CA050020280A00209802002000
:104A5000880C00203C01002010B5FCF789F90F48B4
:104A6000018821F0020101800C49183109880C4AA3
:104A7000928E1144094A3432118008490C390A884F
:104A800042F001020A80011D0A884FF6ED531A40D8
:104A90000A80018841F01201018010BD0C04004021
:104AA0004004002006480188491C89B20180B1F504
:104AB0007A7F04D34188491C4180002101807047DE
:104AC000140700200F4810B5016841F00101016092
:104AD00041680D4A1140416001680C4A1140016073
:104AE000016821F480210160416821F4FE014160E8
:104AF0004FF41F018160FFF7C7FE05494FF00060CA
:104B0000086010BD001002400000FFF8FFFFF6FE35
:104B100008ED00E02DE9F0412F4D28884FF000040A
:104B2000000629D5FCF7A4FA2C4A2D48072317784C
:104B3000C8262C49012F22D02B4FB7F806C0BCF154
:104B4000000F3ED0B0F80CC04CF0080CA0F80CC020
:104B5000B0F806C02CF4006CA0F806C0886820F0FD
:104B600004008860FC801370CE8700204FF49661AB
:104B7000401C80B28842FBD32C80BDE8F0811B4FE3
:104B800097F800C0BCF1010F0FD0BCF1020F11D09B
:104B9000B0F806C04CF4006CA0F806C0886840F07D
:104BA0000400886005203870DDE7B0F80CC04CF0D8
:104BB000080C03E0B0F80CC04CF0100CA0F80CC0CE
:104BC000F0E70B4F3C70C78847F40067C7808868E0
:104BD00040F004008860C6E7102C0140F306002076
:104BE000280A00209802002034090020F406002042
:104BF00011070020704700002DE9F0434FF080407E
:104C0000018A21F001010182AC48007800287CD1A2
:104C1000AB4FF87B002878D1AA48406C322874DC6E
:104C2000A9488068DFF8A4924104A94DB9F80400AE
:104C30004FF0000403D4401CA9F8040028E1002828
:104C400074D02978012611B1012912D017E1494603
:104C5000B0F5BE7FFAD92E70CC718C71EC702C72CD
:104C6000287A0A18401CC0B2147228720F28F7D391
:104C700005E1B9F802204946824201D9EE7100E00F
:104C8000EC7192488A7908300F2A15D2CB79082B1B
:104C90000BD2C3F10708EB7912F800C003FA08F34E
:104CA00063441354CA79521CCA71CA79082A03D1C1
:104CB0008A79521C8A71CC7199F80610C8460F295E
:104CC00073D10D21FCF73EF9A881010A6970C0B2C9
:104CD000A87088F8064098F816208A4265D198F89E
:104CE0001510814261D198F80BC07A490323022242
:104CF0007948BCF1000F10D0BCF1010F02D0BCF11B
:104D0000020F14D080F86A2000E0CBE091F800C0D8
:104D10002CF00C0C0CF1080C0FE080F86A6091F894
:104D200000C02CF00C0C0CF1040C06E0A9E080F89B
:104D30006A3091F800C04CF00C0C81F800C098F873
:104D40000C10B6EB111F04D180F86E4087F8464076
:104D50000EE0B2EB111F04D180F86E6087F8466058
:104D600006E0B3EB111F03D180F86E2087F84620D0
:104D70000B0717D001F00F01012901D0022915D02E
:104D800080F86C602C7198F80D102A7906FA02F3FD
:104D90000B406B71082A44D2DFE802F00B12431972
:104DA000242F363D80F86C40ECE768E080F86C20FA
:104DB000E8E713B180F8704033E080F8706030E0CD
:104DC00013B180F850602CE080F8504029E023B106
:104DD00080F8656087F8036123E080F8654087F814
:104DE00003411EE023B187F8F54080F84D4018E0FC
:104DF00087F8F56080F84D6013E013B180F86860C3
:104E00000FE080F868400CE013B180F8666008E0BD
:104E100080F8664005E013B180F8676001E080F833
:104E20006740521CD2B22A71082AAED398F80E10ED
:104E30002A4A8B0705D587F8F16080F864605681AF
:104E400004E087F8F14080F864405481C90702D03B
:104E500080F8294001E080F8296098F8111000F8E6
:104E60006D1FC2781E48012A1ED001B3012921D02E
:104E70004FF48051A0F876101A493C200870A9F828
:104E80000240A9F80440B9F80210491CA9F8021020
:104E9000B9F80210B1F5FA7F04D940F2F511A9F87A
:104EA00002102C70BDE8F08344F21C71E2E74FF46D
:104EB0000051DFE741F25551DCE70000F306002026
:104EC000980200203C01002000100140700C0020DE
:104ED0008C060020B8040020880C0020280A00203E
:104EE00020050020F00600202DE9F05FFDF710FA04
:104EF0008E4D2888A5F10406C0070AD0308820F01E
:104F000008003080288820F00900288001F0ACFDDE
:104F1000D9E02888DFF81892DFF81882864C8007DD
:104F20001AD5B9F8001041F00101A9F80010B8F83D
:104F30000000804914315030088028884FF6F9511C
:104F400008402880308840F004003080FFF718F8CF
:104F500084F83C00BDE8F09F2888784F40072888F7
:104F600071D520F004002880FFF70AF894F83C106F
:104F70008142EFD1308820F004003080FDF7A0FBA3
:104F80002078410605D594F84C1094F83B209142C6
:104F9000E0D03978400621F00201397004D5FEF7DF
:104FA000AFFA97F82F7004E094F83C00FDF702FA8E
:104FB0000746DFF880B140F68C2A0BF1180B062F5C
:104FC00047D294F83800B8423ED03846FDF776F91B
:104FD0002078C00716D094F83A0094F8391000F001
:104FE0000302914206D0A17A00F0010001F0010114
:104FF000884215D1FDF7CCFAFBF706FFFDF7F4FB6D
:10500000384689E0FDF7C4FAFBF7FEFEFDF7ECFB3E
:105010003846FDF7DDFA207840F00100207099E76E
:10502000288820F008002880206B810801EBD00040
:10503000504515D2B8F800100844ABF8000030888D
:1050400040F0080003E00DE0308820F008003080D8
:1050500080E7B9F8001041F00101A9F80010DFE77E
:105060005046E7E70007288831D520F0080028805F
:10507000308820F008003080FEF782FF84F83C0082
:10508000FDF71EFB387820F00200387020784006CB
:1050900004D5FEF735FA97F82F5004E094F83C0059
:1050A000FDF788F90546062D08D294F83800A84285
:1050B000B5D0FDF76DFAFBF7A7FE2AE02048C188BE
:1050C00041F04001C180BDE8F05FFDF76DBBC00657
:1050D000288825D520F010002880308820F0100086
:1050E000308097F838000C2802D2401C87F838002E
:1050F000387840F002003870FEF702FA97F82F5027
:10510000787884F8390094F83800A84287D0FDF701
:105110003FFAFDF769FB2846BDE8F05FFDF758BA96
:105120004EF2BE110840288014E700001004004031
:1051300000040040240400403C0100204004002002
:10514000280A00202DE9F04F514F85B0388820F013
:10515000010038804E480026103006804D4CDFF8A4
:1051600038A14FF0010894F85C0042F63029C107DD
:1051700074D072B64948816941F4007181618169D6
:1051800041F4806181614FF40040FEF75FFE444DC1
:1051900000212846FBF796FB00212846FBF788FBF9
:1051A000DFF800B100215846FBF782FB00213E48A2
:1051B000FCF7FAF92846FBF7A1FC5846FBF79EFCE2
:1051C0004FF46020CDE902068DF8056000968DF859
:1051D00010808DF8048069462846FBF721FD0123E5
:1051E0001A460F212846FBF76CFD01212846FBF7E4
:1051F0005FFB00204946401C80B28842FBD3284612
:105200002E600121FBF79CFD28688007FCD524480F
:105210004C30006894F85C1021F001012144A1F8A1
:105220005000FBF759FB62B6FEF776F847F690613F
:10523000AAF8001094F85C00401CC0B284F85C002E
:105240000C2822D212491431A1F80080388840F08D
:105250000100388005B0BDE8F08FFFE7134920F06A
:105260000100085A12490880114945F658000839CA
:1052700008800F4847F25801001F01800C49202088
:105280000C390880AAF80090D4E70320A070E1E769
:1052900000080040400400202C080040001002409C
:1052A000002401400028014008000240908B0008C3
:1052B000202C01400029018802D041F0800101E04A
:1052C00021F080010180704710B50A884B88CC8896
:1052D0001A438B8823431A430B891A434B898989C4
:1052E0001A430A43A0F8442010BD002101804180E8
:1052F0008180C1800181418181817047002981883D
:1053000002D041F0010101E021F0010181807047EC
:105310000029018802D041F0010101E021F00101E2
:1053200001807047002930F8441F02D041F4004149
:1053300001E0C1F30E010180704700004B4910B538
:10534000884202D10121C41486E0B0F1804F09D017
:10535000474988420DD101210220FEF799FD002125
:10536000022064E001210846FEF792FD00210120A1
:105370005DE04049884206D101210420FEF788FD06
:105380000021042053E03C49884206D10121082035
:10539000FEF77EFD0021082049E03849884206D109
:1053A00001211020FEF774FD002110203FE0344958
:1053B000884206D101212020FEF76AFD002120202D
:1053C00035E03049884202D10121441444E02E499D
:1053D000884202D10121CC043EE02C49884202D10E
:1053E00001210C0538E02A49884202D101214C05EF
:1053F00032E02849884206D101214020FEF748FDCD
:105400000021402013E02449884206D10121802058
:10541000FEF73EFD0021802009E0204988420AD1A4
:10542000841501212046FEF733FD00212046BDE80A
:105430001040FEF72DBD1A49884202D101210C040B
:105440000AE01849884202D101214C0404E01649BF
:1054500088420AD101218C042046FEF731FD204606
:10546000BDE810400021FEF72BBD10BD002C01400F
:105470000004004000080040000C00400010004004
:105480000014004000340140004C01400050014035
:105490000054014000180040001C00400020004063
:1054A000004001400044014000480140002A828938
:1054B00001D00A4300E08A438281704730B5028CF4
:1054C00022F001020284028C8388048B22F0020203
:1054D00024F073050C882C430D8915434A882A4310
:1054E000114DA8420BD0114DA84208D0104DA84232
:1054F00005D0104DA84202D00F4DA8420DD122F088
:1055000008054A8923F440732A4322F004058A8857
:105510002A438D891D43CB892B4383800483C9880B
:105520008186028430BD0000002C0140003401401F
:10553000004001400044014000480140028B22F03D
:1055400008020A430283704770B5028C22F01002F1
:105550000284028C8488038B0D8823F4E6464FF680
:10556000FF7303EA052535430E8922F0200203EA82
:10557000061616434A8803EA02123243104EB0421E
:1055800002D0104EB04215D122F080064A8924F490
:10559000406403EA0212324322F040068A8803EA9A
:1055A000021232438E8903EA86062643CC8903EA37
:1055B0008404344384800583C9880187028470BDD4
:1055C000002C014000340140028B4FF6FF7322F49F
:1055D000006203EA012111430183704770B5028C18
:1055E00022F480720284028C8488838B0D8823F0DD
:1055F00073031D4322F400730E894FF6FF7202EA13
:1056000006261E434B8802EA03233343104EB04262
:1056100002D0104EB04215D123F400664B8924F419
:10562000405402EA0323334323F480668B8802EA62
:10563000032333438E8902EA06162643CC8902EA05
:105640000414344384808583C9888187038470BDB2
:10565000002C014000340140828B22F008020A43F2
:105660008283704770B5028C22F480520284048CCD
:105670008288838B0D8823F4E6464FF6FF7303EA96
:105680000525354324F400560C8903EA04343443D9
:105690004E8803EA06362643094CA04202D0094C44
:1056A000A04205D122F480448A8903EA821222436F
:1056B00082808583C988A0F84010068470BD0000F0
:1056C000002C014000340140828B4FF6FF7322F41E
:1056D000006203EA012111438183704701858282C0
:1056E0007047828822F07002828082880A4382801A
:1056F0007047A0F84010704730B502881B4B1C4C17
:1057000098420DD0A0420BD0B0F1804F08D0194D77
:10571000A84205D0184DA84202D0184DA84203D186
:1057200022F070054A882A43154DA84206D0154D2F
:10573000A84203D022F44075CA882A4302808A888E
:1057400082850A88028598420AD0A04208D00E4A73
:10575000904205D00D4A904202D00D4A904201D1AC
:10576000097A01860121818230BD0000002C0140B0
:10577000003401400004004000080040000C0040DC
:10578000001000400014004000400140004401406F
:10579000004801404FF6FF71818000210180C180E7
:1057A0004180017270470029018802D041F0020156
:1057B00001E021F00201018070470029018802D038
:1057C00041F0040101E021F0040101807047000074
:1057D000204810B590F82010026801F01F001E4903
:1057E00051F820001D490242086802D040F4803080
:1057F00001E020F48030086019484FF00002807901
:105800004106184824D4184903880C88E31A9CB22E
:1058100001230F2C08D30C8804808468042C03DD3A
:10582000124C2478022C05D0427F012A06D0098828
:10583000418010BD4377C2770A8842804288098838
:10584000891A89B240F21A629142F2D3C37710BD2D
:10585000427710BDD0050020D48F000898020020A8
:10586000280A0020500C0020FC060020F30600202F
:105870002DE9F04FDFF8B8B16A48DFF8AC91DFF8F6
:10588000ACA190F80EC0BBF91A70BBF91C60BBF953
:105890001850BBF96C10BCF1070F48D2DFE80CF0D0
:1058A0008D041A30485E7600D9F800208284DAF838
:1058B0000020C284828CC38CA7EB820212B2A6EBBA
:1058C00083034A431BB2594342F3CF2241F3CF2310
:1058D000D11870E0D9F800204284DAF80020C284A0
:1058E000428CA5EB820213B2C28C4B43A6EB820220
:1058F00012B243F3CF24514341F3CF23E11814E014
:10590000D9F80020C284DAF800204284C28C438C8B
:10591000A6EB820212B2A5EB83031CB24A43614399
:1059200042F3CF2341F3CF24191949420AB244E08C
:10593000D9F800208284DAF800204284828C438CDB
:10594000A7EB820212B2A5EB83034A431BB2594371
:1059500042F3CF2241F3CF24111914E0D9F80020EB
:105960004284DAF800208284428C838CA5EB820288
:1059700012B2A7EB83034A431BB242F3CF2459432D
:1059800041F3CF22A11849420BB216E0D9F800200A
:10599000C284DAF800208284C28C838CA6EB820257
:1059A00012B2A7EB83031CB24A4342F3CF236143F5
:1059B00041F3CF22991849420CB2BBF91E50594607
:1059C00005F21E56A64201DACE8306E0A5F21E5568
:1059D000A54201DDCD8300E0CC83B1F9204004F283
:1059E0001E55954201DA0D8406E0A4F21E5494423D
:1059F00001DD0C8400E00A84B1F9222002F21E5479
:105A00009C4202DAABF8224008E0A2F21E529A420F
:105A100002DDABF8222001E0ABF82230417B81733C
:105A2000BDE8F08F980200203C2401403C28014052
:105A3000200500202DE9F04704466448654D002606
:105A400002786348022AB0F9301004D0082A7DD0C9
:105A5000092A7CD0B6E0C27B022A02D1B0F84020ED
:105A600052B1A4F8421069810423B5F908101A460E
:105A70000020FEF74FFF9CE05749DFF86081496A3C
:105A80000F14E7808068410216D5B4F9020040F295
:105A9000DA21884277DD40F26A41884205DD00BFA5
:105AA0000823B4F942101A4648E0A0F2DA20FAF7C7
:105AB000B4FC00224A4B52E0C0F3C001C0F3002006
:105AC000DFF8209181420CD1D8F8440040F2BA416D
:105AD000884258DD40F66A118842E1DCA0F2BA4003
:105AE00010E041480078C00611D5D8F8440041F2D2
:105AF0002431884247DD41F2D4718842D0DCA0F5E0
:105B000098502438FAF789FC00224B4627E03748A2
:105B100090F87010012903D090F86F00012832D15D
:105B2000B4F9020041F6DC6188422CDD42F2341106
:105B300088420DDDB4F9421020231A460020FEF7FA
:105B4000E9FEA4F84200002819DB1EE033E037E04C
:105B5000A0F5F050DC38FAF760FC0022244BFAF78D
:105B6000C8FB0E22FAF734FCFAF78EFC00B2C0F53F
:105B7000804078438013A4F84200002F05DCA4F88D
:105B8000426002E0FFE7A4F84270B4F84200194F07
:105B9000E880D8F844107964A7F84C0000F07EFB48
:105BA000B7F84E00688198F80A000028388F00D1B5
:105BB0004042288106E01048B0F87C00688100E08F
:105BC00069812E8184F84060BDE8F087F3060020EB
:105BD0009802002060000020200500203C010020E9
:105BE0000000794000C09240D4060020880C0020BC
:105BF00000C08240C80800203C0A00202DE9F04186
:105C0000B1F9025000232B241522854203DAB1F9A1
:105C10000000BDE8F081B1F9AE50854202DDB1F976
:105C2000AC00F6E701EB8205B5F90250854201DDD3
:105C3000134600E01446E21852085D1CAA42F1D156
:105C400001EB8205B5F90230834206DA35F9026CC0
:105C500035F9044C31F9221006E01E4631F9224094
:105C6000B5F90630B5F90410801B091BC517891159
:105C7000AD0345EA90458703A1FB070CCA1702FB59
:105C800007C201FB05219A1BD317FAF74BFA000A4A
:105C900040EA0160001900B2B0F5804FB9DB43F66D
:105CA000FF70B6E770B5134C40F2244529462046F4
:105CB00000F03EF800281BD0204600F0C7F8294627
:105CC000204600F01DF80C4C00212046FBF76CFC30
:105CD0002046FBF7E7FCC0F164000849C0B2042885
:105CE000087201D900F046F9BDE87040FBF720BD0D
:105CF00070BD000000380140580002405C060020E2
:105D00000A0A01219140C943018070470029818915
:105D100002D041F4005101E021F40051818170472B
:105D2000002A828A01D00A4300E08A4382827047B7
:105D300030B501F01F0201240025C1F3421304FA1B
:105D400002F2012B0FD0022B0FD0838A4FEA1121D0
:105D50000088134204FA01F400EA040001D000B103
:105D60000125284630BD8389F0E7038AEEE710B5A8
:105D7000C1F3421301F01F040121A140012B07D000
:105D8000022B07D01430002A026805D00A4304E031
:105D90000C30F8E71030F6E78A43026010BD0000CF
:105DA00030B50446008A85B00D464CF6FF710840B8
:105DB000E98801432182A1894EF6F3100140A888A9
:105DC0002A8910436A890A431043A081A08A4FF6AA
:105DD000FF410840A9890143A1826846FEF77CF88B
:105DE0001948844201D1039800E00298A18909046E
:105DF00000EBC00101EB0010296801D5490000E06B
:105E00008900B0FBF1F06422B0FBF2F109010B094B
:105E10006FF018056B4300EB8300A3891D044FF05E
:105E2000320306D503EBC000B0FBF2F000F0070030
:105E300005E003EB0010B0FBF2F000F00F000843A8
:105E4000208105B030BD0000003801408088C0F3DB
:105E500008007047F8B501210920FEF725F8012157
:105E60008803FEF721F810258DF803502020ADF8A7
:105E700000001A4E03248DF8024069463046FCF7B4
:105E80008FF916490C31086820F0200008601820AE
:105E90008DF803004020ADF800008DF802406946FF
:105EA0003046FCF77DF948208DF803008020ADF8DE
:105EB000000069463046FCF773F98DF8035028015D
:105EC000ADF800008DF8024069463046FCF768F9ED
:105ED00001210420FCF7B6F9F8BD0000000C0140D8
:105EE00030B585B0FFF7B6FF00244FF4E1300090E5
:105EF000ADF808400C201D4DADF80440ADF80A0087
:105F0000ADF80640ADF80C4069462846FFF748FF5B
:105F100025208DF8100004208DF811008DF8124016
:105F200001208DF8130004A8FDF786FC012240F241
:105F300024412846FFF71BFF01212846FFF7E6FE14
:105F4000FBF720FC012280212846FFF7E9FE012211
:105F500040212846FFF7E4FE012202210448FBF716
:105F6000B5FBFBF70FFC05B030BD00000038014069
:105F70004400024070B51D4D00242878432834D1D8
:105F80006878462831D1A878502807D0512805D004
:105F9000812803D0892801D0212826D1144E707180
:105FA000E9787172A81C891CFBF704F8B072717A49
:105FB000294409793182884217D106F10E0001780F
:105FC00041F0020101700B48016841F020010160BD
:105FD000317A0948002204E02B5D03552A55641CE0
:105FE000E4B28C42F8D38078707170BD88070020CD
:105FF0005C0600200C0C0140BA0B002070B51D207F
:10600000FDF7F9FBFDF77CFA1D20FDF70AFC1548AA
:1060100090F82F10144D0623144C85F8381090F882
:106020003B1095F83B201143012A04D0022A07D0E7
:10603000042A0AD010E0827A8A420DD0007B09E05F
:10604000027D8A4208D0807D04E0827F8A4203D0AC
:1060500090F82000884200D12370002085F840008D
:1060600070BD0000400400203C010020F306002029
:106070000B4800214180A0F1B0018A898280CB8940
:106080001A44C2800B8A1A4402814B8A1A44428104
:10609000898A1144818143F6FF71C18170470000F4
:1060A000EC010020084940F61C72B1F90C00904246
:1060B00002DA00F59F7005E041F2E302904201DD53
:1060C000A0F59F70C88170476000002038B5134864
:1060D000C16941F00401C1611E208DF80000022059
:1060E0008DF801008DF8020001248DF80340684608
:1060F000FDF7A2FB0A4984200880094947F6906011
:106100002C3108800020091F0880054914310C80BB
:10611000091F0880081F048038BD000000100240DD
:106120000008004030B420491E4A45788B7A114659
:1061300092F83B4091F83910AC4218D14BB1037939
:10614000994202D04379994201D140791AE080798D
:1061500009E08379994202D0C479A14202D182F840
:106160002F3011E0407982F82F0030BC7047C5789D
:10617000AC42FAD16BB1C379994202D0037A994209
:1061800005D1007A82F82F0030BCFEF765BC407A5A
:10619000E9E7437A9942E2D00479A142DFD0007A5C
:1061A000E1E70000400400203C010020FEE7000081
:1061B0002DE9F0470446007F012868D13548E18881
:1061C0000288511A89B2072916D30088E080B4F9F1
:1061D000000044F2DD414843401346F6D96148438C
:1061E0008013A060401000B2A0814FF08051B1FB3D
:1061F000F0F0FAF70DF92061B4F90C6096B1B4F93A
:1062000002104DF6B05048430014A082B4F9047057
:106210004DF6B05207FB02F24FEA2245E58204D464
:10622000024603E00020E08330E0424212B22283C3
:10623000002D01DB2B4600E06B421BB2DFF85890CB
:10624000638398464FF4804AB24208DAFAF7D7F8E7
:106250002169F9F7AAFFFAF7FEF8801304E0002994
:1062600001DA484600E05046E083B04509DA2846A6
:10627000FAF7C5F82169F9F798FFFAF7ECF88013F7
:1062800004E0002F01DA484600E050462084BDE8D3
:10629000F0870000FC06002000C0FFFF10B5224878
:1062A000234C01782148022905D1C17B022902D162
:1062B000B0F8401029B1008EA4F84E0000202087CD
:1062C00010BD90F846101A48B0F8440000B239B337
:1062D00018490978C1F3810101291BD002291CD07A
:1062E000154900BFFBF7B4FD1149A4F8400080B286
:1062F000483101F071FAB4F94C00B4F94A20414236
:106300005143891324F8381FB4F9101048438013FF
:10631000E08210BD0849D839E4E707496C39E1E764
:1063200005496C31DEE70000F306002098020020EA
:10633000C8080020B804002008890008034800218C
:1063400080F82A10C183018770470000C808002028
:1063500010B504000B462D4AC3F1000028D5644255
:10636000002B12DAA04207DA214600F027FA32F8B1
:106370001000C0F5404041E00146204600F01EFA02
:1063800032F8100000F5004038E0A34208DA214658
:10639000184600F013FA32F8100000F540402DE0E6
:1063A000204600F00BFA32F81000C0F5803025E0EE
:1063B000002B12DAA04207DA214600F0FFF932F88A
:1063C000100000F5804019E00146204600F0F6F983
:1063D00032F81000C0F5004010E0A34208DA214670
:1063E000184600F0EBF932F81000C0F5804005E0E7
:1063F00053B1204600F0E2F932F81000B0F5004F3A
:1064000001DDA0F5803010BD002010BD9C8B000880
:1064100040438013494300EBA13000220302002BCC
:1064200014DDB3F5001F01DC802001E04FF40050C3
:1064300093FBF0F1014401EBD1714910814206D088
:10644000521CD2B20846062AF2D300E00021C8004E
:1064500000B2704702E008C8121F08C1002AFAD132
:1064600070477047002001E001C1121F002AFBD1D4
:10647000704700002DE9F047A44CA5482188028808
:10648000511A89B20F297DD30088A4F13C052080E0
:10649000288F08B1401E28872B789E4AC3F38100BD
:1064A00001281DD0022820D0D18B98489A4FDFF8C0
:1064B0006C92407E0026B1F5926F1DD8142819D336
:1064C00078206076F88840F01000F88040F266602E
:1064D000A88123F001002870D67389F8006015E0C8
:1064E000D08B00EB4000C00302E0D08B8C494843C6
:1064F000010CDAE7401C04E0B1F5DB6F06D310B104
:10650000401E607602E043F001002870B5F90200F9
:10651000B5F914304143C3EBC303C1F38F31C3F367
:10652000D10303EB510109B2A9829046D28B4FF0FF
:1065300080535043B5F91620C0F38F30C2EBC2022E
:10654000C2F3D10202EB500000B2E882AA6A4243D1
:106550001213EA6293FBF2F22A63724A1080A26875
:106560000A44A260E1680144E160207C401CC0B2A2
:106570002074072806D942F3CF002883C910698305
:10658000E66000E0BFE0A66041F6C80126748842DC
:1065900004DD298B644AB2FBF1F1E981C11789035B
:1065A00041EA9041800342F69B420023F9F7BAFD8D
:1065B000A88456482A78A0F13C005C49B0F906004E
:1065C000930700FB01F14FEA2141C2F3810215D587
:1065D000012A07D0022A0BD04FF268514143091417
:1065E000A18011E049F68C4250430014A0801FE0C6
:1065F0004CF6183141430914A18025E0012A0DD041
:10660000022A17D0A0806984494948430014E083D6
:10661000FBF73EFA47480088C0B143E04AF65C32D7
:1066200042431214A2804BF62C225043001468847B
:10663000E183EDE74DF2AC5141430914A1804EF2E4
:106640007C414143091469843B49DEE795F8200009
:1066500000BB88F80F6089F80060B5F91A00A0F552
:106660000C519F39B1F56E7F18D8617FF42912D98A
:106670003249E8802E4AA1F8460050430014A88011
:10668000A1F84400FF2085F8200081F828002C495B
:106690003C20087006E0491C617703E0607F08B188
:1066A000401E6077B5F91A10B4F91E0081420EDD64
:1066B000A07E7D2809D9F88840F00800F88021489C
:1066C000017821F0020101700EE0401C06E0A0F20A
:1066D0003D10814208DAA07E10B1401EA07603E092
:1066E000F88820F00800F880B5F9181060690844AF
:1066F0006061217E491CC9B221761F2903D940114E
:10670000A88366612676BDE8F0870000F4040020C7
:10671000FC06002098020020280A0020F306002032
:1067200030330100DC09002074E8260BCC0E010098
:1067300048850100FE060020D0450100880C00209D
:10674000F0060020CA050020024941F68B3088621D
:1067500070470000B804002070B5164C062520785C
:10676000062825D2DFE800F003080E141A2112488B
:10677000FAF75EFC012016E00F48801DFAF758FC7E
:10678000022010E00C480C30FAF752FC03200AE01B
:1067900009481230FAF74CFC042004E0064818308F
:1067A000FAF746FC0520207070BDFAF761FC2570F1
:1067B000257070BDF4060020E0890008090A05D0A4
:1067C000B0FBF1F0FF2800D9FF2070470020704790
:1067D000D0E90021C368521A5A4301EBA23181600B
:1067E00041607047B0F90020B0F90210B0F90630EE
:1067F000521A5A4301EBA231818041807047000058
:1068000030B5494B188849498A89801A85B2484869
:10681000484A0F2D047801F14C001DD31D888D814D
:10682000117A090713D5022C01D0434912E0434DD8
:10683000B0F90210B5F90050A94205DC02DA01F105
:10684000020108E0458007E0A1F1020103E0022C0B
:1068500002D13B4909884180B0F840101D88691A6F
:1068600089B29C2949D31988A0F84010916A002365
:10687000B1F5804F31DB3349896CB1F5405F2CDDD8
:10688000314940F26665B1F91010A94212DD43F6B4
:106890009915A94202DB40F2333108E040F233356A
:1068A000A1F26661694343F2333591FBF5F1A0F83B
:1068B000441001E0A0F844302449B2F806510978A8
:1068C000C1F381012DB100BFB0F8441001F21E5197
:1068D0001CE092F84620022A10D0A0F84430022C86
:1068E00001D0A0F84430B0F95C10B0F9443001F1A7
:1068F00014029A420DDAA0F85C2030BD012901D0C3
:106900000229E1D1B0F8441001F23331A0F844106B
:10691000E5E703F11402914203DD1439A0F85C109D
:1069200030BDA0F85C3030BDFC0600201400002013
:10693000F306002098020020B6040020B4040020D2
:10694000B00400203C01002020050020B8040020F5
:106950002DE9FC4101210220FDF78EFA01211920C9
:10696000FDF7A2FA01213C48FBF76CFC4027ADF88B
:10697000007003248DF802400420384D8DF8030088
:1069800069462846FBF70CFCE001ADF800008DF8E5
:1069900002401C208DF8030069462846FBF700FCE6
:1069A0004FF4E0712846FBF782FCA815ADF8000013
:1069B0008DF8024010208DF8030069462848FBF747
:1069C000EFFB4FF4A060FCF769FF1D208DF8040079
:1069D00001268DF8056000258DF806508DF80760BA
:1069E00001A8FCF729FF1F498C2008801D494FF69C
:1069F000FA702C3108806E20091F08801948143065
:106A00000680184808300780164920310D80154A45
:106A1000D020121D1080134A45F2F3001832108066
:106A20000A1F45F2500010800E4A4FF6FF703832B0
:106A30001080121D1080121D108041F21B10088062
:106A400000F012F8FBF7B0FE064810300580001F7A
:106A50000480BDE8FC810000000C1A000010014019
:106A6000000C01400004004070B51D20FCF7B8FE8A
:106A70002A4D40212846FBF711FC8400802128463E
:106A8000FBF70CFC44EA4004A9152846FBF706FC7A
:106A90000443E0B2224C84F83C00FBF78BFC054633
:106AA000052805D91F48C18841F04001C18001E097
:106AB00084F838501C48007A000703D594F8380051
:106AC0001A490D5C4FF6FA702063E062A0626062C2
:106AD0002062E061A0611648606300206064A064E9
:106AE00084F83F0084F84000FBF712FCA07AFF28EE
:106AF00011D0022084F83D000E4800882066284608
:106B0000FCF7B4F8207820F001002070BDE8704058
:106B10001D20FCF77BBE0120ECE7000000100140C7
:106B20003C010020280A002098020020A0930008C1
:106B3000DCFF0500240400402DE9F0434E484F4996
:106B400002880B889A1A92B20F2A69D309880180A9
:106B50004B49098B027D00EB42029180017D491C6B
:106B6000C9B2017508295BD3002404752246017D52
:106B700000EB4103491CB3F90430C9B202EB6302D4
:106B800012B201750829F2D33E4904753E4B4A8082
:106B900044800E789D895FEAC67C40F638694FF0E4
:106BA000030714D0A2F22B5C42F6E858C44520D368
:106BB000A1F1020C26F00204ACF8002047750C701D
:106BC00040F22B54A24211DA45F004021EE046F0D6
:106BD00001060E704A4507DD45F001029A8126F054
:106BE00002020A70477519E0447517E045F0020289
:106BF0000CE04A450CDA8775427D12B1521E42758F
:106C00000CE046F002020A7025F007029A8105E0C6
:106C1000B30703D5837D2BB15B1E837540888880C5
:106C2000BDE8F08342F6AA239A4222DAB1F9043091
:106C30002BB941F2CD05AA4201DA4480EEE7134CAC
:106C4000920302EB843241F67244B2FBF4F214B2C6
:106C500040F2333502464480AC4200DA5580B2F946
:106C60000240E41A04F5A374B4F5237FD6D8438018
:106C7000D4E74FF48043FAE7BC0A0020FC0600206A
:106C800098020020CA050020280A0020C8F1FFFF52
:106C90002DE9F0416D4CDFF8B8E14FF0000594F8B4
:106CA0003410C80706D094F938104B42002958DD3B
:106CB0000E4657E0674884F83750A4F84250664AB9
:106CC00090F8380084F840001586CEF80450CEF8CD
:106CD0000850624E40F26663CEF80C50A4F87C3047
:106CE00036F810005E4E768830444FF6FF7606EA9E
:106CF000800024F8300B4FF0806044F8040CA3208F
:106D0000208460845810A084E38440F69910208584
:106D1000580060854FF48050A08541F23330E08503
:106D200041F26660208641F69910608641F6CC40BB
:106D3000A0864FF40050E08642F23330208742F2C2
:106D40006660608742F69910A08742F6CC40E087E3
:106D500082F89D5041F00100207184F84450BDE854
:106D6000F0811E4694F937004242002801DD0746B3
:106D700000E01746F61B012E0BD0002800DB024670
:106D80005FFA82F684F8380094F84F00012805D0A5
:106D900041E0002900DA1946CEB2F3E794F9393020
:106DA0005942002B01DB184600E0084694F93A20CE
:106DB000C7B25042002A01DB944600E08446BC453D
:106DC00008DD002A00DA0246D7B2002B00DA0B46B3
:106DD000D8B207E0002B00DA0B46DFB2002A00DB56
:106DE0001046C0B204EB4000B0F9501004EB47006D
:106DF00030F9502F11444910018084F84F5084F825
:106E00003E5084F83D5084F83C5084F83B5084F860
:106E10003A5084F8395004EB46007546B0F95000FA
:106E200024F8420FBEF80410C82309B26422FDF70B
:106E300071FD6860E968401AA9680844A860B5F95E
:106E400000104843C013E860608788E73C0A0020D0
:106E5000B80500203C01002098020020B2930008F1
:106E600060000020F0B4544890F83410C90776D080
:106E7000524990F84030002291F838108B426FD080
:106E80004F4CA0F872204F4DE65C04468E4294F9B8
:106E9000374002D0EE5C8E420FD1641C64B280F8A1
:106EA0003740EB5C8B4202D1641C80F8374090F98C
:106EB00037300F2B1BDD0F2317E0434DEE5C434DA6
:106EC0008E4202D0EE5C8E4211D1641E64B280F814
:106ED0003740EB5C8B4202D1641E80F8374090F95A
:106EE00037406FF00E039C4201DA80F83730324BA6
:106EF00090F83F50393390F83740EC5490F83F30D9
:106F00005B1CDBB280F83F30062B01D380F83F20BA
:106F100090F9394090F93B309C420ED190F93D40B8
:106F2000A3420AD190F93A4090F93C309C4204D1F6
:106F300090F93E40A34200D1012280F84F201F4A21
:106F400080F8401090F937501378214A012D0DDD5B
:106F500014465E07A46804D544F0080403E028E062
:106F600015E024F00804946080F83510B5F1FF3F77
:106F70000ADA5B07936802D523F0080301E043F0C7
:106F80000803936080F83510F0BCFBF7C1B990F8A6
:106F90004F1001290DD1B0F8721043F60953491C66
:106FA00089B2A0F87210994203D9A0F8722080F833
:106FB0004F20F0BC704700003C0A00203C0100203C
:106FC000949300089A930008A6930008AC930008D5
:106FD0009802002030B52049204AB1F86A30108864
:106FE000C01A80B20F2836D31088A1F86A001C4D51
:106FF00000204FF000432A5C940903D00124B4EB35
:10700000921F24D1D20622D0164A52F820201268AC
:10701000134C123434F81040224201EB000494F96E
:10702000722008D00A2A04DB0A6823FA00F42243FB
:1070300008E0521C09E012F10A0F05DC0A6823FA85
:1070400000F4A2430A6002E0521E84F87220401C41
:10705000C0B21128CFD330BDD0050020FC060020DF
:10706000A08F0008A09000082DE9F00779497A4820
:107070000A8903889A1A92B2082A74D30088088170
:10708000A1F12C0042890AB1521E4281734A92F842
:107090002820802A67D302F03F020A70C2890AB111
:1070A000521EC281B1F90620902A0CDB8A46FF2AC3
:1070B00009D08146C089002855D16948002300784D
:1070C000092805D005E0BDE8F007624800F096B950
:1070D0000823644A92F8EA500DB143F00403624871
:1070E000817AC90701D043F00203D2F808C05FEAF1
:1070F0000C5101D543F00103176800215B4EFC03DE
:1071000002D596F8654004B18021C4885FEA4468DE
:1071100001D541F040015FEA845801D541F02001DA
:107120005FEAC47801D041F01001007A400701D530
:1071300041F008014E480078C00701D041F0040139
:10714000A00601D541F001010020012D00D1082049
:1071500096F8705085B992F84620022A04D0012A88
:1071600005D03AB108E072E040F0030004E040F0DE
:10717000020001E040F001007A0701D440F0200055
:10718000CCF3C0020025CCF3002C624502D13A07B3
:1071900000D4042596F86F20012A01D145F001059D
:1071A000344A0027BC4612783E46C2F38102012AC7
:1071B00004D0022A04D0032A04D004E0022602E00C
:1071C000042600E010262C4A64060ED5214C1C34FF
:1071D0002478240609D51478640606D4274A40F694
:1071E000CC44926D6243140C05E0B2F8AE2040F638
:1071F00099146243940B4FF008088AF80A804FF004
:1072000061088AF80B808AF80C308AF80D108AF829
:107210000E008AF80F508AF81070270A4B4083F04E
:107220006901414069408AF8117079408AF812403A
:10723000614052468AF813C071408AF81460517553
:107240004FF4C871A9F80E10FF20AAF80600BDE897
:10725000F0077047B8060020FC060020D00500208B
:10726000F306002098020020280A0020880C002045
:107270001C090020B80400203C010020EC0700207D
:107280004E48816941F0FC0181614FF4A060FCF738
:1072900005FBFBF717FBFCF765FCF9F787FCFCF730
:1072A0005BFAFDF73DFAFFF753FBFCF79BF9FFF79D
:1072B000DBFBFBF779FA424D4FF40050A5F81601BD
:1072C000FEF70EFE00214FF4FA5340F2EE220020AA
:1072D000401C80B29842FBD3491C89B29142F6D33C
:1072E0003848002680F87260F9F7F6FAF9F79CFF43
:1072F000FCF768FCF9F76AFEFEF7E8FE1022324957
:107300003248F8F740FF324C334FE08820F040001D
:10731000E0803048017821F020010170FA20F881E6
:107320004FF49670E887FFF70FFA2C492C48FCF7CA
:10733000C6FB2C48FCF7E8FB2B48416A88472B48E2
:10734000416B8847FEF7FAFF2948FAF79DFB294968
:107350004220C8802849C8603E71E088E0812089C9
:10736000208260896082FAF793FEFAF7F5FDFFF755
:1073700081F8FFF7E1FB00F0FDF9FFF72BFE00F0CD
:10738000CBFFFEF725FAFAF753FCFBF78DFCFFF76E
:1073900037FAFCF76FFEFBF7AFF8FBF7E1F800F008
:1073A0007BF8FFF761FE1248FAF736FA00F06EFA42
:1073B000FDF7FAF9FAF79EFBCFE700000010024054
:1073C0009802002020050020880C002010060020D4
:1073D000280A00203C010020F00600209808002028
:1073E00068080020F803002034000020D8000020A6
:1073F000A8090020180700202C040020F0B523491C
:107400000278B0F9064000231F4E31F81210FF2C0D
:1074100018D0B0F904701E4DBC4231DA00EBE4071D
:1074200004F00704BF7AA7408478FFB23CB190F81B
:1074300001C0ACF1010C64451FDA3C061DD455F8BF
:1074400022200DE056F82220116012498A79521C40
:10745000D2B28A71022A02D38370C3808B71F0BDCD
:1074600011608178491CC9B2817042789142F6D38B
:107470008370C188491CC180F0BD56F82220EFE717
:1074800055F822201160F4E780910008B28F0008BF
:10749000289100088C060020F0B561486149B0F8D9
:1074A0006C200B889A1A92B29C2A7BD30988A0F888
:1074B0006C105D495D4F91F82A1001F0070297F8B2
:1074C0004610022A00D1491E594C80F83E104FF058
:1074D0000203E2884FF00001550401D5012236E095
:1074E000A489E50601D5062231E0250701D5082249
:1074F0002DE0550603D44F4D2D78AD0601D504225D
:1075000025E0150501D5072221E0150601D50A223F
:107510001DE0950601D50C2219E0150701D50B22B7
:1075200015E0550701D4D50501D510220FE0D50689
:1075300001D505220BE0650703D4A50701D4E407B4
:1075400002D080F86E3007E0920403D5032280F861
:107550006E2001E080F86E10374A384C92F820E037
:10756000324A251FD2F808C02D4AB2F87060721C4A
:1075700092B2BEF1000F0DD02CF4000CC7F808C079
:1075800090F86E70B7B11E2F1AD090F86F200AB322
:1075900025E007E04CF40006BE60A0F870200A2A3F
:1075A00001D22360F0BD142A01D22B60F0BDA0F8F7
:1075B0007010F0BD2B60A0F8701080F86F10F0BD57
:1075C000642E04D2A0F87020322AEED3E9E7A0F8A6
:1075D0007010EAE77F1C80F86F70A0F8701090F8C8
:1075E0006F20012A10D0002AE9D0B0F87060761C14
:1075F000B6B2A0F870601E2ED7D323603C2EDED921
:10760000521E80F86F20D2E7B0F87020521C92B260
:10761000A0F870202360C82AD1D980F86F10C6E77F
:10762000D0050020FC060020880C002098020020D5
:10763000280A00203C010020B8040020141C01404E
:10764000F0B54548B0F84810491C89B2A0F8481078
:1076500002297DD341490024A0F848400A78404BD4
:10766000042A5BD04FF48041082A0BD0A0F10C0211
:10767000B2F900208A4200DA1146B3F980208A422A
:1076800000DA1146374A92698A4200DA11B2418221
:1076900082881D8AC2EB8502334D12B22D78C5F364
:1076A00081062D4D42F231667243B5F97650921241
:1076B0006A431213C26086681546C6EBC60642F3DB
:1076C000D102F60202EBA6328260C66C1644C66492
:1076D000B0F850707F1CBFB2A0F85070B7F5806F43
:1076E00004D3B6120682A0F85040C464891AC26A54
:1076F000A2EB421606EB0616A6EBC21640F2551296
:107700004A4306EB4202466A32444262B3F93030E1
:10771000B2EB034F06DD1A04426206E01349B1F9E9
:107720000410AFE7002A00DA4462C162104990F801
:107730003D2091F838108A420DD080F83D10B0F805
:107740004210A0F84410B0F84010A0F8421000E039
:1077500001E0A0F84050F0BD20050020F306002015
:1077600098020020200C0020B80400203C0C0020CF
:107770003C01002015481649B0F85A200B889A1A87
:1077800092B20F2A20D30988A0F85A10B0F900103D
:1077900041F6515251438913A0F86C100D494FF432
:1077A00080420B78A0F10C01022B06D1B1F9003018
:1077B000934202DA1B1D0B8000E00A800021A0F832
:1077C000601020F85C1F42807047000020050020F8
:1077D000FC060020F30600204FF6FF7202EA80024A
:1077E00010F4404315480ED0B3F5804F14D0B3F5D4
:1077F000004F4FEA122216D0C2F5807330F81330D2
:107800005B424B8005E0120A30F812304B80C2F523
:10781000807230F812000FE0120AC2F5807330F85F
:1078200013304B8005E030F81230C2F580725B42B5
:107830004B8030F812004042088070479C8D000851
:10784000104A518A908AD28A16384639A2F111021A
:1078500000D54942002A00DA52421144002800DAD9
:1078600040420844084943F6284300B2B1F93620A3
:107870005A43921340F2D733584302EBA030C886E4
:10788000704700009802002020050020F0B59049C4
:1078900090480A8903889A1A92B23E2A1ED3008819
:1078A000088101F138004FF4FA63428A9A4202D209
:1078B000521C428200E04382874A92F82220802AAA
:1078C0000CD302F03F020A70B1F90620402A06DB11
:1078D000FF2A04D0C2883AB1521EC280F0BDBDE872
:1078E000F0407B48FFF78ABD428A9A42F6D3077878
:1078F0004FF0010E3A074FF0FF055BD5847A40F256
:10790000DC52630708D444F004038372C28081F818
:107910000BE081F80AE04CE04378072B05D0032BFD
:1079200003D0052B01D0062B07D1660605D444F001
:1079300040038372C280052239E0654A5FEA437CD6
:1079400002F138024FF42076127A0DD55FEAC26C4C
:107950000AD45FEA446C07D442F0100202723A067D
:1079600028D4C680192222E0DF0709D0970707D460
:10797000670605D442F002020272C680042216E0B5
:107980009F0709D5170707D4670605D442F00802F8
:107990000272C68003220AE01B070BD5530709D4E5
:1079A000630607D442F004020272C6800B22CA7238
:1079B0008A72CD80494AB2F92230B2F91A7003F2C4
:1079C0003D140022A74200DB0276414E444C06F1F2
:1079D0003806A479B6895FEAC46C06F101064FF453
:1079E000C874B6B213D58681B6F57A7F05D9017A07
:1079F00021F0800101728281F0BD037A1E06FBD462
:107A0000828143F080020272C480112035E09F42DF
:107A100016DA037E052B13D28681B6F5487F04D98A
:107A20008281027A22F040020272027A5606E3D480
:107A30005B1C037642F040020272C48002201CE00C
:107A4000284B1C89C4F3C006C4F3002740F2EE247F
:107A5000BE4216D11E78360713D4427E012ACBD1FE
:107A6000428BB2F5167F02D2521C4283F0BD827A5D
:107A700042F002028272C4800F20C8728872CD80E8
:107A8000F0BD93F80D714FF40046012F18D1164F39
:107A900041F6583C7F6C674512DD83F80CE1134BCF
:107AA0001E60C38AA34202D25B1CC382F0BD4FF4A6
:107AB000FA73C3801C23CB728B72CD80C282F0BD5F
:107AC000C2820A4883F80C21001F0660F0BD000046
:107AD0009C060020FC060020D0050020B8040020F1
:107AE000280A0020980200203C01002014080140D0
:107AF0002DE9F05FFE48FF49DFF8FCA3007E0A1D78
:107B0000131D012850465AD030F85A4F0C80418836
:107B10001180BAF85E001880F84DF94C49F2CD3268
:107B2000B5F91E106183B5F9200043F6CC4C01EB8A
:107B3000400050430014A083B4F92230B4F920600F
:107B400000FB03F201FB062242F38F326282B4F99A
:107B5000167007FB0CF7BF1340F2333C704302FB77
:107B60000CF201FB130007EBA232E28240F38F30EC
:107B7000A082B4F91810E34FC1EBC10141F3D10168
:107B800001EBE000E04E2083786C306031693046D4
:107B90008847DE49308948800846FDF74BFFDFF80B
:107BA000709301264FF0020B99F800004FF0000887
:107BB00008280CD0618F2182042840D01AE030F8C8
:107BC000604F0C8041881180BAF86400A3E7D14867
:107BD00090F93710491C02292FD890F8741019B168
:107BE000B4F85A00208205E0618F2182A4F85A106F
:107BF00080F87460B4F91410B4F90A00C64AF9F7B1
:107C00004DFCE062BAF91611884204DDC248E16217
:107C1000027C91408162BA4847F2A3014C38DFF8F8
:107C2000FCE290F800C04A00BCF1000F0BD0BCF1A0
:107C3000010F80F8008058D12BE0608FD2E7686A8E
:107C40000014E06278E0B5F91EC08C44944509D870
:107C5000B5F920C08C44944504D8B5F92250294484
:107C6000914242D9A0F80280B7F8AE204146B2F561
:107C7000C87F01D8467007E0B2F5487F02D880F887
:107C800001B001E0032242708AF80F1089F8001059
:107C900023E0B5F91EC08C44944509D8B5F920C03D
:107CA0008C44944504D8B5F92250294491421CD9FA
:107CB000B7F8AE10B1F5C87F01D8467007E0B1F54E
:107CC000487F02D880F801B001E003214170A0F89C
:107CD00002808AF80F8089F80080BEF8061041F40F
:107CE0000061AEF80610FAF729F999F800000428A7
:107CF00022D0894AB4F91210B4F90800303AF9F7E1
:107D0000CDFB42F6F821A062884200DBA162844DDF
:107D1000A06A2860E06A68602846FCF711F87E4F88
:107D2000287C443F01280FD0A06A38607D48017844
:107D3000C9070DD040690CE0B87A10B17A48A0624A
:107D4000E5E74FF4AF70FAE768693860A86900E0CA
:107D5000E06A786070484438FCF766F9684D684915
:107D600035F8100F3C39FFF737FDDFF89491A9F192
:107D70004C09D9F81010C9F86C10B5F91010B86892
:107D8000B5F9122000FB01F4FB68504303FB1244D9
:107D900044F38F3703FB0100AF8740F38F34EC8748
:107DA000624D28466F80AC80FEF702FA287F09F109
:107DB000140501282FD0604241104DF6B3504743BF
:107DC0003A1469802A808B18A9F80440A9F8063073
:107DD000891AA9F808108AF80C80B9F904305446B9
:107DE0004946002B00DD2673B1F90600002802DDAC
:107DF000227B921C2273B9F90820002A02DD217B24
:107E0000091D2173217B072924D2DFE801F0231CFF
:107E1000361A211F34004548B0F9203059424A1023
:107E20006A80B0F91E004DF6B35148430014288013
:107E3000A9F804301318A9F80630101AA9F8080098
:107E4000C9E7667306E084F80DB003E0032100E0A3
:107E500004216173DFF8A890354E364F99F8001071
:107E60000129617B0BD0072941D2DFE801F0E6FE52
:107E7000FDFCFBFAF9000521EBE70621E9E70729FC
:107E800035D2DFE801F0DA041B637A9AB0000146CC
:107E90001846FBF7FBFD2860B5F90200B5F90010A4
:107EA00043F2046201445143090C5043A4F85A10B0
:107EB000000CA4F85C00A4F85E8028E1404201B206
:107EC000504200B2FBF7E2FD2860B5F9020043F230
:107ED00004614143090CA4F85A10B5F90010084494
:107EE00043F204614843000CA4F85C0024E0A4E0E1
:107EF000A8090020342C0140980200202005002011
:107F0000600000203C0100202C040020E803002039
:107F1000F30600203C0A002098080020280A0020D0
:107F2000000A00201C090020A2FEFFFFDC0900203F
:107F30000024014000280140A4F85E8015E130468D
:107F4000F8F792FE01231A4607216BE01946104606
:107F5000FBF79CFD2860A4F85A80B5F90200B5F93A
:107F6000001043F2046201445143090C5043A4F849
:107F70005C10000CA4F85E0026E15942404209B2B0
:107F800000B2FBF783FD2860A4F85A80B5F902001F
:107F900043F204614143090CA4F85C10B5F90010E8
:107FA000084443F204614843000C39E13046F8F7D5
:107FB0005BFE01231A46052134E01146FBF766FDFE
:107FC0002860B5F9020043F204614143090CA4F8AA
:107FD0005A10A4F85C80B5F90010084443F204611B
:107FE0004843000C47E1504201B2584200B2FBF74F
:107FF0004DFD2860B5F90200B5F9001043F20462A6
:1080000001445143090CA4F85A105043A4F85C8071
:10801000000CA4F85E005EE13046F8F725FE01236F
:108020001A4606213846F8F71FFE01213046F8F7B8
:1080300091FD01213846F8F78DFDB44EB9F80800DE
:108040004D463080B9F80A007080B9F81000B08051
:108050003046F9F72DFCB4F85A00F188084405E0E1
:1080600017E1EBE0BCE08DE05DE030E0A4F86000FB
:10807000B4F85C0031890844A4F86200B4F85E00EA
:1080800071890844A4F86400317EA148012978D0A0
:1080900034F85A1F018061884180A18881809C4901
:1080A000028808310A8042884A80808888809848FF
:1080B000896A0830884795F83E0000287ED0F8F796
:1080C000D7FF15F83E0F401E2870BDE8F09F01460F
:1080D0001846FBF7DBFC2860B5F9020040F6815139
:1080E000484381136980B5F9000040F6815250433E
:1080F00080130A18A2F68152524252082880114475
:10810000A4F85E20A4F85C100844A4F85A000021EA
:108110003046F8F71FFD00213846F8F71BFD012314
:108120001A4606210BE7404201B2504200B2FBF76B
:10813000ADFC2860B5F9020040F681514843801338
:108140006880B5F9001040F68152514389134218F6
:10815000A2F68152524252082980A4F85E201044AF
:10816000A4F85A000844A4F85C0000213046F8F74F
:10817000F1FC00213846F8F7EDFC01231A460521F1
:10818000DDE6B4E019461046FBF780FC2860B5F93F
:10819000020040F68151484381136980B5F900001F
:1081A00040F68152504380130A18A2F6815252427F
:1081B00052082880A4F85A20114400E09AE0A4F85C
:1081C0005E100844A4F85C0000213046F8F7C2FCB9
:1081D00000213846F8F7BEFC01231A460721E5E6E0
:1081E0005942404209B200B2FBF750FC2860B5F991
:1081F000020040F68151484380136880B5F90010B1
:1082000040F68152514389134218A2F681525242DC
:1082100052082980A4F85A201044A4F85C000844AD
:10822000A4F85E0000213046F8F794FC002138469F
:10823000F8F790FC01231A460621B7E61146FBF732
:1082400025FC2860B5F9020040F6815148438013AF
:108250006880B5F9001040F68152514389134218E5
:10826000A2F68152524252082980A4F85C201044A0
:10827000A4F85A000844A4F85E0000213046F8F73C
:1082800069FC00213846F8F765FC01231A460521F0
:10829000C2E6504201B2584200B2FBF7F7FB286039
:1082A000B5F9020040F68151484380136880B5F962
:1082B000001040F68152514389134218A2F68152B0
:1082C000524252082980A4F85C201044A4F85E00B1
:1082D0000844A4F85A0000213046F8F73BFC00217E
:1082E0003846F8F737FC01231A46072194E634F89C
:1082F000601FCFE607480088A0F5D04168393FF4F9
:10830000E4AEBDE8F05FF9F767BD0000A809002002
:108310002C000020182C01402DE9F041904C914890
:10832000B4F85A100288511A89B20F296FD3008805
:10833000A4F85A008C480088DFF83082C0074FF05C
:1083400000054FF0010741D0874AD4E90C102432D0
:108350001388B1EB530F02D21288511A08444FF41C
:10836000F371884200D208468149B1FBF0F0616C9C
:10837000C1F35101084406466064F8F74EF8002244
:108380007C4BF7F7B6FF4FF040427B4BF7F7B1FF5E
:108390000E22F8F71DF8F8F777F8A4F8A40094F87F
:1083A0006500401CC0B284F86500082834D36C48CE
:1083B00098F84620001F03789A4201D00270458049
:1083C0006E4A13786E4A23B1458021E06564A56446
:1083D00058E0D8F89410A1F5FA618E4211DD616D74
:1083E0008B1C9E4205DDB0F902100A290DDA491CEA
:1083F00006E08E4205DAB0F90210002908DD491EB8
:108400004180B0F902000A2802DB177001E0A2E007
:108410001570666584F865505A484FF4A542017896
:10842000C1F38101012949D002294AD044F687715C
:108430002181A4F8A020B0F9243089B24B439B13CA
:10844000A4F89C30B0F90E0000237043B0FBF1F0AB
:10845000A16CC0F3D100C1EBC101C90200EB9130A6
:10846000A064F017810341EA9641B003F7F75AFE82
:10847000B4F8A210C1EBC101C902C00800EB9130F1
:10848000A4F8A200616CA06E0844A06694F86C2069
:10849000521CD2B284F86C20082A05D3C008A4F874
:1084A0006E0084F86C50A5663748384EC3885A066B
:1084B00033D498F80F20022A06D02CE043F204515E
:1084C000B6E744F24621B3E7B26840F69916B242E5
:1084D00021DD94F8382094F88660B2420CD084F8FC
:1084E000862094F83D2002F00106C2F34002964235
:1084F00002D1A4F8825004E0B4F88220B2F5966F5D
:1085000005D2B4F88200401CA4F8820005E043F0D4
:108510008002C28001E0A4F88250114894F83F30F4
:10852000B0300C2B01D2C57400E0C774174A0F4C51
:1085300041F2482692F83C20B4F8824041F2504C77
:108540000C2B0AD3B14208DB012A06D0614502DDBB
:10855000002C00D18774BDE8F0818574FBE7000032
:108560003C010020FC06002000040040980200208E
:108570004564BD0100209C40133B3340E6030020CE
:10858000E7030020B8040020280A0020200500206E
:108590002DE9F041384C394E394F207841F23331D2
:1085A000C2074FF000050CD0A28962B394F907000E
:1085B000002800DA4042C0B2032829D240F2AE704F
:1085C0002AE0A570E5732F4AE571A58192F838304D
:1085D000237220F00800A18040F0020020703D8648
:1085E0007560B560F560916C490005D041F6846115
:1085F000A18140F010002070C0B240F00100207056
:108600006574BDE8F081658120F01000207015E0F0
:10861000042803D240F6510060810FE0052802D201
:1086200040F69910F8E740F6CC42062803D3072815
:1086300001D3082801D2628100E0618197F89D0092
:1086400098B9B088102301B2B4F90A003622FCF7B9
:1086500061F97060F168401AB1680844B060B6F919
:1086600000104843C013F0603886388E10B10120E6
:10867000A070C6E7A570C4E73C0C00207C06002073
:10868000980200203C0100202DE9F041554C26784D
:10869000F0077CD05448217A544D90F8380081423C
:1086A0007BD0534A2346DFF84CC1575C93F90E2028
:1086B00093F90730874203D01CF80170874213D129
:1086C00046F002065B1C26705BB2E3711CF80110D9
:1086D000814201D15B1CE37194F90710062901DD89
:1086E0000621E171521C1CE0434F17F801C0434FB3
:1086F000844503D017F801C0844513D126F0020643
:108700005B1E26705BB2E371795C814201D15B1E16
:10871000E37194F907306FF005018B4200DAE171E3
:10872000521EA273207294F907108A1C042A02D9DF
:1087300041F68462A2812C4A012912780ADD2B4B72
:1087400056079B6802D543F0080301E023F00803B5
:10875000AB606070B1F1FF3F09DA5107A96802D53B
:1087600021F0080101E041F00801A9606070F9F70B
:10877000CFFDA078012810D121488068A3280CDA09
:1087800094F90700022803DD0220E07105E01EE0F5
:108790006FF00101884200DAE171A089002630B152
:1087A000401E0004000CA08101D1E671A673E87B95
:1087B00004280CD0B5F93010512341220020FCF7D9
:1087C000A9F82886002802D1E07B10B1A670BDE888
:1087D000F0810C4806700C480670207820F00100EB
:1087E0002070F4E73C0C00203C010020980200209F
:1087F000949300089A930008A6930008AC9300088D
:108800002005002010070020F3060020743F713D72
:108810009B3BED396238F436A13565343F332A325B
:10882000273133304C2F722EA32DDF2C242C722BAA
:10883000000000361C070038AA0A003AAA0A003CC9
:10884000CC0C003ECC0C0040380E0042380E0044E8
:10885000380E0046380E0048380E004AC711004C4A
:10886000C711004EC7110050C7110052C711005464
:10887000C7110056C7110058C711005AC711005C34
:10888000C711005EC7110060C7110062C711006404
:10889000C7110066C7110068C711006A00000036E2
:1088A000220200388E03003AB005003CD207003E99
:1088B000F4090040160C0042380E00445B100046DC
:1088C000C71100483313004A9F14004C9F14004EF8
:1088D0000B16005077170052771700547717005681
:1088E000771700587717005A7717005C7717005EE4
:1088F00077170060771700627717006477170066B4
:10890000771700687717006A000000368E0300387A
:108910006606003A3E09003C160C003EEE0E004092
:10892000111100423313004455150046C11600488A
:108930002D18004A9919004C051B004E711C00505F
:10894000271D0052DD1D0054931E0056491F00587C
:108950000020005AB520005C6C21005E22220060DD
:10896000D82200628E23006444240066FA24006842
:10897000B025006A00000034000000360000003816
:108980000000003A0000003C0000003E00000040F3
:1089900000000042000000440000004600000048C3
:1089A0000000004A0000004C0000004E0000005093
:1089B0000000005200000054000000560000005863
:1089C0000000005A0000005C0000005E0000006033
:1089D0000000006200000064000000660000006803
:1089E000441458585870111158585870411158581B
:1089F000487011144858587014115848587033135F
:108A0000005695130054B61300525A140050FD142A
:108A1000004EA115004C4516004A761600486C170A
:108A2000004672180044BA190042741B0040911DA0
:108A3000003EB420003C9F22003AE122003853233C
:108A400000368B240034812500322B27003020286B
:108A5000002E5829002CB02A002A9B2C0028D22D49
:108A600000267C2F00242631002202330020FD3412
:108A7000001E5C37001CCC3C001A873E0018BE3F2D
:108A8000001600400014004000120040001000409A
:108A9000000E0040000C0040000A004000080040AA
:108AA00000060040000400400002004000000020DA
:108AB0000072002000700020006E0020006C00207A
:108AC000006A00200068002000660020006400208A
:108AD0000062002000600020005E0020005C00209A
:108AE000005A0020005800200056002000540020AA
:108AF0000052002000500020004E0020004CA32017
:108B0000004AA320004847210046EB210044EB2106
:108B100000428F2200408F22003E7A24003C7A24BB
:108B2000003A66260038512800343D2A0030702D66
:108B3000002CA33000287A34002451380020CC3C8B
:108B4000001C0040001800400014004000100040CD
:108B5000000C00400008004000040040000000003D
:108B600001020304050005000102030401040003DF
:108B700005020000F001000036010000F8000000CE
:108B8000BA0000007C0000007C0000007C000000B7
:108B9000411414111114441114144111000029003E
:108BA00052007B00A400CC00F5001E0147017001BB
:108BB0009901C201EA0113023C0265028E02B6026B
:108BC000DF020803300359038203AA03D303FB0324
:108BD00024044C0475049D04C504EE0416053E05EA
:108BE00067058F05B705DF0507062F0657067F06C1
:108BF000A706CE06F6061E0746076D079507BC07B3
:108C0000E4070B08320859088108A808CF08F608BD
:108C10001D0944096A099109B809DE09050A2B0AE8
:108C2000520A780A9E0AC40AEA0A100B360B5C0B39
:108C3000820BA80BCD0BF30B180C3E0C630C880CAD
:108C4000AD0CD20CF70C1C0D410D650D8A0DAF0D4E
:108C5000D30DF70D1C0E400E640E880EAC0ECF0E19
:108C6000F30E170F3A0F5E0F810FA40FC70FEA0F15
:108C70000D103010531075109810BA10DD10FF1041
:108C80002111431165118711A911CA11EC110D129F
:108C90002E12501271129212B312D412F412151332
:108CA0003613561376139613B713D713F6131614F9
:108CB0003614561475149414B414D314F2141115F4
:108CC00030154E156D158C15AA15C815E715051626
:108CD000231641165F167C169A16B716D516F2168D
:108CE0000F172C17491766178317A017BC17D9172A
:108CF000F51711182E184A18661881189D18B918FA
:108D0000D418F0180B19261942195D1978199219FF
:108D1000AD19C819E219FD19171A311A4C1A661A39
:108D2000801A991AB31ACD1AE61A001B191B331BA5
:108D30004C1B651B7E1B971BAF1BC81BE11BF91B44
:108D4000121C2A1C421C5A1C721C8A1CA21CBA1C13
:108D5000D21CE91C011D181D301D471D5E1D751D0F
:108D60008C1DA31DBA1DD01DE71DFD1D141E2A1E3E
:108D7000401E571E6D1E831E981EAE1EC41EDA1E98
:108D8000EF1E051F1A1F2F1F451F5A1F6F1F841F1D
:108D9000991FAE1FC21FD71FEC1F002000006400E8
:108DA000C9002D019201F7015B02C002240389036F
:108DB000ED035204B6041A057F05E3054706AB062A
:108DC0000F077307D7073B089F0802096609C909FF
:108DD0002D0A900AF30A560BB90B1C0C7F0CE20CFF
:108DE000440DA60D090E6B0ECD0E2F0F900FF20F36
:108DF0005310B41015117611D71138129812F812B9
:108E00005813B81318147714D61435159415F31590
:108E10005116B0160E176B17C91726188318E018CD
:108E20003D199919F519511AAD1A081B631BBE1B80
:108E3000181C731CCD1C261D801DD91D321E8A1EB8
:108E4000E31E3B1F921FEA1F41209820EE20442181
:108E50009A21EF2145229922EE2242239623E923EB
:108E60003C248F24E22434258525D72528267826FE
:108E7000C82618276827B72706285428A228EF28CD
:108E80003D298929D629222A6D2AB82A032B4D2B60
:108E9000972BE12B2A2C722CBB2C022D4A2D912DC5
:108EA000D72D1D2E632EA82EEC2E302F742FB82F09
:108EB000FA2F3D307F30C030013141318131C13135
:108EC00000323F327D32BA32F73234337033AC3352
:108ED000E73322345C349534CE3407353F3577356B
:108EE000AE35E4351A3650368536B936ED3620378C
:108EF00053378637B737E937193849387938A838BA
:108F0000D738053932395F398B39B739E2390D3AFB
:108F1000373A603A893AB23ADA3A013B283B4E3B5B
:108F2000733B983BBD3BE03B043C263C483C6A3CE1
:108F30008B3CAB3CCB3CEA3C093D273D443D613D8D
:108F40007D3D993DB43DCE3DE83D013E1A3E323E69
:108F5000493E603E763E8C3EA13EB53EC93EDC3E7B
:108F6000EF3E013F123F233F333F433F513F603FBE
:108F70006E3F7B3F873F933F9E3FA93FB33FBC3F40
:108F8000C53FCD3FD53FDC3FE23FE83FED3FF13FFE
:108F9000F53FF93FFB3FFD3FFF3FFF3FFF3F000035
:108FA000E7382C35002020EF2037202333202620DF
:108FB00021000080020004000800100000020004EC
:108FC0000008040000020004000800100020004017
:108FD000008004000000008000000040000000202D
:108FE0000000001000000008000000040000000263
:108FF0000000000100008000000040000000200090
:109000000000100000000800000004000000020042
:10901000000001000080000000080140000C014039
:10902000000C0140000C0140000C0140000C01400C
:10903000000C0140000C01400010014000100140F4
:1090400000100140001001400010014000100140DC
:1090500000100140001001400014014004080140CC
:10906000040C0140040C0140040C0140040C0140BC
:10907000040C0140040C0140040C014004100140A8
:10908000041001400410014004100140041001408C
:109090000410014004100140041001400414014078
:1090A00008080140080C0140080C0140080C014070
:1090B000080C0140080C0140080C0140080C01405C
:1090C000081001400810014008100140081001403C
:1090D000081001400810014008100140081001402C
:1090E000081401400C0801400C0C01400C0C01401C
:1090F0000C0C01400C0C01400C0C01400C0C01400C
:109100000C0C01400C1001400C1001400C100140EF
:109110000C1001400C1001400C1001400C100140DB
:109120000C1001400C14014010080140100C0140CB
:10913000100C0140100C0140100C0140100C0140BB
:10914000100C0140100C01401010014010100140A3
:10915000101001401010014010100140101001408B
:1091600010100140101001401014014000000000D8
:1091700000000000000000000000000000000000EF
:1091800014080140140C0140140C0140140C01405F
:10919000140C0140140C0140140C0140140C01404B
:1091A000141001401410014014100140141001402B
:1091B000141001401410014014100140141001401B
:1091C0001414014000000000000000000000000036
:1091D0000000000000000000FFFFFF0F0FFFFFFF77
:1091E000FFF0FFFFFF0FFFFFFFFFF0FF0FFFFFFF8D
:1091F000FFF0FFFFFF0FFFFFFFF0FFFF0FFFFFFF7D
:10920000FFF0FFFFFF0FFFFFFFFFF0FFFFFF0FFF6C
:10921000FFFFFFF0FFFFFF0FFFF0FFFF0000004028
:1092200040000000000400000040000000000400B6
:1092300040000000000400000040000000040000A6
:109240004000000000040000004000000000040096
:109250000000400000000004000000400004000086
:109260000000008080000000000800000080000076
:1092700000000800800000000008000000800000DE
:1092800000080000800000000008000000800000CE
:1092900000000800000080000000000800000080BE
:1092A0000008000000000020200000000002000074
:1092B000002000000000020020000000000200006A
:1092C000002000000002000020000000000200005A
:1092D000002000000000020000002000000000024A
:1092E000000000200002000000000060600000009C
:1092F00000060000006000000000060060000000A2
:109300000006000000600000000600006000000091
:109310000006000000600000000006000000600081
:10932000000000060000006000060000008002004F
:1093300004000800100000020004000804000002FD
:10934000000400080010002000400080040000001D
:10935000FF7FFFFFFDFFFFFFFBFFFFFFF7FFFFFFAB
:10936000EFFFFFFFFFFDFFFFFFFBFFFFFFF7FFFF2B
:10937000FBFFFFFFFFFDFFFFFFFBFFFFFFF7FFFF0F
:10938000FFEFFFFFFFDFFFFFFFBFFFFFFF7FFFFFDD
:10939000FBFFFFFF010203040500020304050001B7
:1093A0000304050001020500010203040405000195
:1093B000020355050010AA1A55250030AA3A0000EC
:1093C000AA0A55150020AA2A5535FF3FEC9300083C
:1093D0000000002024070000E4060008DC940008D8
:1093E00024070020DC09000064640008450204062C
:1093F000082D010203040405440607080913552B30
:109400001B086904190A12152A40061908019F133E
:10941000853D1B08A9041AA50401251702060405A9
:109420000103148020FF8BAA0A02019C15AA0A5589
:109430001500085920AA2A5535FF3F0729030105C1
:1094400004060203127C1573FFFF04FF80800101F4
:1094500025025F6402130A13D16712081201100C6F
:109460000504060203010103070505280B01020399
:10947000040206070303040C3D0706040509191F2F
:10948000191904310506064BAA1A024B381E026947
:1094900010312E40FD3969260211042F405F020C65
:1094A00026405B262ACD55155515123902017F033A
:1094B00016D0071AFF01013B0261AA6C080108A837
:1094C0000916C491220312100A17401C12600A16D2
:0C94D000901B014913E567020008000032
:020000040800F2
:10FC00004A46545A594D46312D4E3330202020203B
:10FC1000050406020301AA0AAA0AAA0AAA0AAA0A4B
:10FC2000AA0ADE3F00100000FF0131000201664613
:10FC300000400040513800400040004000400101B9
:10FC400000400040FF387B257B257B25FF003333B8
:10FC50000201401F00016626B81E6626FFFFFFFF57
:10FC6000FFFF01010100010000000300000200008D
:04FC70000000AA5591
:04000005080000ED02
:00000001FF
